:020000040800F2
:1000000000070020F5040008912F0008492F000880
:10001000712F0008492F0008692F0008F704000815
:10002000F7040008F7040008F7040008853F0008FB
:10003000F7040008F7040008F7040008F7040008B4
:10004000F7040008F7040008F7040008F7040008A4
:10005000F7040008F7040008396B0008616B00081A
:10006000896B0008B16B0008D96B0008F704000821
:10007000F7040008F7040008F7040008F704000874
:10008000F7040008F7040008F7040008FD2E000834
:10009000292F0008392F0008F7040008016C000818
:1000A000F7040008F7040008F7040008F704000844
:1000B000E96C0008F7040008F7040008F7040008DA
:1000C000F7040008F7040008F7040008F704000824
:1000D000F7040008F7040008D56C0008F7040008CE
:1000E000656C0008F7040008F7040008F70400082E
:1000F000F7040008F7040008F7040008F7040008F4
:10010000F7040008F7040008F7040008F7040008E3
:10011000F7040008F7040008F7040008F7040008D3
:10012000F7040008F7040008F7040008F7040008C3
:10013000F7040008F7040008F7040008F7040008B3
:10014000F7040008F7040008F70400082961000814
:10015000F7040008F7040008F7040008F704000893
:10016000F7040008F7040008F7040008F704000883
:10017000F7040008F7040008F7040008F704000873
:10018000F7040008F7040008F7040008F704000863
:10019000F7040008F7040008F7040008F704000853
:1001A000F7040008F7040008F7040008F704000843
:1001B000F7040008F7040008F7040008F704000833
:1001C000F7040008F7040008F7040008F704000823
:1001D000F7040008F7040008F7040008F704000813
:1001E000911800080000000000000000000000005E
:1001F00053B94AB9002908BF00281CBF4FF0FF318E
:100200004FF0FF3000F074B9ADF1080C6DE904CE89
:1002100000F006F8DDF804E0DDE9022304B07047E1
:100220002DE9F047089D04468E46002B4DD18A42A9
:10023000944669D9B2FA82F252B101FA02F3C2F1DC
:10024000200120FA01F10CFA02FC41EA030E94406D
:100250004FEA1C48210CBEFBF8F61FFA8CF708FB8E
:1002600016E341EA034306FB07F199420AD91CEB66
:10027000030306F1FF3080F01F81994240F21C8198
:10028000023E63445B1AA4B2B3FBF8F008FB1033E0
:1002900044EA034400FB07F7A7420AD91CEB040415
:1002A00000F1FF3380F00A81A74240F207816444E5
:1002B000023840EA0640E41B00261DB1D44000236A
:1002C000C5E900433146BDE8F0878B4209D9002DCE
:1002D00000F0EF800026C5E9000130463146BDE858
:1002E000F087B3FA83F6002E4AD18B4202D38242C2
:1002F00000F2F980841A61EB030301209E46002D71
:10030000E0D0C5E9004EDDE702B9FFDEB2FA82F2C5
:10031000002A40F09280A1EB0C014FEA1C471FFA23
:100320008CFE0126200CB1FBF7F307FB131140EA0A
:1003300001410EFB03F0884208D91CEB010103F1D7
:10034000FF3802D2884200F2CB804346091AA4B299
:10035000B1FBF7F007FB101144EA01440EFB00FE6D
:10036000A64508D91CEB040400F1FF3102D2A645D2
:1003700000F2BB800846A4EB0E0440EA03409CE771
:10038000C6F12007B34022FA07FC4CEA030C20FA1E
:1003900007F401FA06F31C43F9404FEA1C4900FA3E
:1003A00006F3B1FBF9F8200C1FFA8CFE09FB1811BB
:1003B00040EA014108FB0EF0884202FA06F20BD92E
:1003C0001CEB010108F1FF3A80F08880884240F27E
:1003D0008580A8F102086144091AA4B2B1FBF9F0C2
:1003E00009FB101144EA014100FB0EFE8E4508D9BD
:1003F0001CEB010100F1FF346CD28E456AD9023842
:10040000614440EA0840A0FB0294A1EB0E01A14226
:10041000C846A64656D353D05DB1B3EB080261EB94
:100420000E0101FA07F722FA06F3F1401F43C5E96E
:10043000007100263146BDE8F087C2F12003D840A4
:100440000CFA02FC21FA03F3914001434FEA1C47E6
:100450001FFA8CFEB3FBF7F007FB10360B0C43EAD8
:10046000064300FB0EF69E4204FA02F408D91CEB88
:10047000030300F1FF382FD29E422DD90238634486
:100480009B1B89B2B3FBF7F607FB163341EA034126
:1004900006FB0EF38B4208D91CEB010106F1FF3875
:1004A00016D28B4214D9023E6144C91A46EA00466C
:1004B00038E72E46284605E70646E3E61846F8E6FE
:1004C0004B45A9D2B9EB020864EB0C0E0138A3E747
:1004D0004646EAE7204694E74046D1E7D0467BE728
:1004E000023B614432E7304609E76444023842E7A0
:1004F000704700BF02E000F000F8FEE772B6374830
:1005000080F30888364880F3098836483649086001
:1005100040F20000CCF200004EF63471CEF2000141
:100520000860BFF34F8FBFF36F8F40F20000C0F23F
:10053000F0004EF68851CEF200010860BFF34F8FF5
:10054000BFF36F8F4FF00000E1EE100A4EF63C71E2
:10055000CEF200010860062080F31488BFF36F8F8D
:1005600005F0AAFA06F08EF94FF055301F491B4AE4
:1005700091423CBF41F8040BFAE71D49184A9142E9
:100580003CBF41F8040BFAE71A491B4A1B4B9A423D
:100590003EBF51F8040B42F8040BF8E7002018495D
:1005A000184A91423CBF41F8040BFAE705F088FA7B
:1005B00006F0BCF9144C154DAC4203DA54F8041B98
:1005C0008847F9E700F042F8114C124DAC4203DACB
:1005D00054F8041B8847F9E705F070BA00070020BB
:1005E000002300200000000808ED00E000010020CA
:1005F000000700204873000800230020BC230020CF
:10060000C023002008590020E0010008E401000890
:10061000E4010008E40100082DE9F04F2DED108AF7
:10062000C1F80CD0C3689D46BDEC108ABDE8F08FC0
:10063000002383F311882846A047002004F02AFDF8
:10064000FEE704F083FC00DFFEE70000F8B501F0F0
:1006500031F905F0D3F930B12B4B00220F211A727A
:100660005A729972DA7205F0ABF9074605F010FA82
:10067000054600283CD1254B9F4239D001339F428B
:1006800039D0234B27F0FF029A4237D1F8B200F05D
:100690001DFF2E4642F2107400F01EFF08B1002428
:1006A000264601F063FD20B1032000F087F8002406
:1006B000264635B1174B9F4203D005F0E1F90024DF
:1006C0002646002005F086F9134B1B6913F480734E
:1006D00018D00EB100F088F801F0C6FA00F068FFFB
:1006E00001F064F9204600F0DBF800F07DF8F9E74E
:1006F0002E460024D0E704460126CDE7064641F207
:100700008834C9E71C46E7E700230020010007B052
:10071000000008B0263A09B00004024008B501F014
:1007200011F9A0F120035842584108BD07B541F224
:100730001203022101A8ADF8043001F021F903B041
:100740005DF804FB38B5302383F31188174803683C
:100750000BB104F06BFD164A144800234FF47A7174
:1007600004F05AFD002383F31188124C236813B15F
:100770002368013B2360636813B16368013B6360D6
:100780000D4D2B7833B963687BB9022001F0DEF997
:10079000322363602B78032B07D163682BB90220C7
:1007A00001F0D4F94FF47A73636038BDC0230020A0
:1007B00045070008E0240020D8230020084B1870CB
:1007C00003280CD8DFE800F008050208022001F039
:1007D000ADB9022001F09CB9024B00225A6070476B
:1007E000D8230020E024002010B501F0BFFC30B178
:1007F000244B03221A70244B00225A6010BD234B55
:10080000234A1C4619680131F8D004339342F9D1C8
:100810006268204B9A42F1D91F4B9B6803F1006339
:1008200003F580339A42E9D205F0FEF805F010F99D
:10083000002001F0D5F80220FFF7C0FF174B1A6C1B
:1008400000221A64196E1A66196E596C5A64596E30
:100850005A665A6E1A6942F000521A611A6922F0F9
:1008600000521A611B6972B64FF0E0233021C3F8C1
:10087000084DD4E9003281F311889D4683F308883E
:100880001047BBE7D8230020E02400200000010827
:1008900020000108FFFF000800230020003802406C
:1008A0002DE9F04F93B0AC4B00902022FF210AA815
:1008B0009D6801F083F9A94A1378A3B9A8480121DA
:1008C00003601170302383F3118803680BB104F0C7
:1008D000ADFCA44AA24800234FF47A7104F09CFCBA
:1008E000002383F31188009B13B19F4B009A1A6079
:1008F0009E4A009C1378032B1EBF002313709A4A54
:100900004FF0000A18BF5360D3465646D146012027
:1009100001F00CF924B1944B1B68002B00F01582F8
:10092000002001F00FF80390039B002B01DA00F088
:1009300087FE039B002BEDDB012001F0E9F8039B10
:10094000213B162BE3D801A252F823F0A909000895
:10095000D1090008650A00080F0900080F090008FE
:100960000F090008EF0A0008BF0C0008D90B0008A7
:100970003B0C0008630C0008890C00080F090008F4
:100980009B0C00080F0900080D0D0008490A00081B
:100990000F090008510D0008B5090008490A0008B0
:1009A0000F0900083B0C00080220FFF7B7FE0028E3
:1009B00040F0F581009B0221BAF1000F08BF1C46F0
:1009C00005A841F21233ADF8143000F0D9FF9EE7CC
:1009D0004FF47A7000F0B6FF071EEBDB0220FFF742
:1009E0009DFE0028E6D0013F052F00F2DA81DFE806
:1009F00007F0030A0D10133605230593042105A8FB
:100A000000F0BEFF17E054480421F9E758480421DC
:100A1000F6E758480421F3E74FF01C08404600F081
:100A2000E1FF08F104080590042105A800F0A8FFE3
:100A3000B8F12C0FF2D1012000FA07F747EA0B0BAF
:100A40005FFA8BFB4FF0000901F004F926B10BF0BF
:100A50000B030B2B08BF0024FFF768FE57E746483F
:100A60000421CDE7002EA5D00BF00B030B2BA1D159
:100A70000220FFF753FE074600289BD0012000F01C
:100A8000AFFF0220FFF79AFE00261FFA86F84046C5
:100A900000F0B6FF044690B10021404600F0C8FFC8
:100AA00001360028F1D1BA46044641F21213022160
:100AB00005A8ADF814303E4600F062FF27E701209C
:100AC000FFF77CFE2546244B9B68AB4207D928469E
:100AD00000F088FF013040F067810435F3E7234BD5
:100AE00000251D70204BBA465D603E46ACE7002EE7
:100AF0003FF460AF0BF00B030B2B7FF45BAF0220D6
:100B0000FFF75CFE322000F01DFFB0F10008FFF699
:100B100051AF18F003077FF44DAF0F4A926808EB0E
:100B2000050393423FF646AFB8F5807F3FF742AFEB
:100B3000124B0193B84523DD4FF47A7000F002FFA9
:100B40000390039A002AFFF635AF019B039A03F83E
:100B5000012B0137EDE700BF00230020DC2400203B
:100B6000C023002045070008E0240020D8230020EF
:100B700004230020082300200C230020DC23002075
:100B8000C820FFF7CBFD074600283FF413AF1F2D09
:100B900011D8C5F1200242450AAB25F0030028BF59
:100BA000424683490192184400F0E2FF019A8048CE
:100BB000FF2101F003F84FEAA8037D490193C8F330
:100BC0008702284601F002F8064600283FF46DAF80
:100BD000019B05EB830537E70220FFF79FFD002807
:100BE0003FF4E8AE00F044FF00283FF4E3AE0027F6
:100BF000B846704B9B68BB4218D91F2F11D80A9B6F
:100C000001330ED027F0030312AA134453F8203CFB
:100C100005934046042205A901F060FA0437804696
:100C2000E7E7384600F0DEFE0590F2E7CDF81480E5
:100C3000042105A800F0A4FE06E70023642104A80F
:100C4000049300F093FE00287FF4B4AE0220FFF777
:100C500065FD00283FF4AEAE049800F0F1FE05906B
:100C6000E6E70023642104A8049300F07FFE002837
:100C70007FF4A0AE0220FFF751FD00283FF49AAEAA
:100C8000049800F0EDFEEAE70220FFF747FD002898
:100C90003FF490AE00F0FCFEE1E70220FFF73EFDDE
:100CA00000283FF487AE05A9142000F0F7FE0421C8
:100CB0000746049004A800F063FE3946B9E73220E5
:100CC00000F040FE071EFFF675AEBB077FF472AE64
:100CD000384A926807EB090393423FF66BAE022055
:100CE000FFF71CFD00283FF465AE27F003074F44D3
:100CF000B9453FF4A9AE484600F074FE04210590C2
:100D000005A800F03DFE09F10409F1E74FF47A70FF
:100D1000FFF704FD00283FF44DAE00F0A9FE0028C7
:100D200044D00A9B01330BD008220AA9002000F00E
:100D30004DFF00283AD02022FF210AA800F03EFFF4
:100D4000FFF7F4FC1C4804F0ABF913B0BDE8F08FDA
:100D5000002E3FF42FAE0BF00B030B2B7FF42AAECB
:100D60000023642105A8059300F000FE0746002833
:100D70007FF420AE0220FFF7D1FC804600283FF42C
:100D800019AEFFF7D3FC41F2883004F089F90598D9
:100D900000F0A4FF464600F05DFF3C46B7E506467E
:100DA00052E64FF0000905E6BA467EE637467CE695
:100DB000DC23002000230020A0860100094A1368DC
:100DC00049F2690099B21B0C00FB01331360064B1A
:100DD000186844F2506182B2000C01FB02001860F6
:100DE00080B27047182300201423002010B5002182
:100DF0001022044600F0E2FE034B03CB206061604A
:100E00001868A06010BD00BF107AFF1F2DE9F041E7
:100E1000ADF5507D0DF13C086EAC40F27512074601
:100E20000D4610A80021C8F8001000F0C7FE4FF4CE
:100E3000C4720021204600F0C1FE02F0B1F8274B39
:100E40004FF47A72B0FBF2F0186093E807000223C7
:100E500084E807000DF5ED702382FFF7C7FF47F622
:100E600005231F49238407A806F054F81D2384F89E
:100E700032310DF2EB2207AB0DF1340C1E4603CEDE
:100E8000664510605160334602F10802F6D13068C1
:100E900010603379137141460122204600F040FF73
:100EA00000230393AB7E029305F11903019380B2F3
:100EB0000123CDE904800093E97E06A3D3E9002352
:100EC000384602F035FC0DF5507DBDE8F08100BFDD
:100ED000AFF300809E6AC421818A46EEE824002098
:100EE000246F00082DE9F0412C4C237ADAB08046BB
:100EF0000D465BBB27A9284601F022F807460028CB
:100F000042D19DF89D60C82E3ED801464FF4A6629E
:100F1000204600F053FE4FF48073C4F8F8314FF4CC
:100F20000073C4F80C334FF44073C4F820343246D5
:100F30000DF19E0104F1090000F01AFE26449DF80F
:100F40009C30777223720BB9EB7E237281220021D1
:100F500006AC27A800F032FE0122214627A801F0A6
:100F60002BF800230393AB7E029305F1190380B2A3
:100F700001932823CDE904400093E97E05A3D3E93A
:100F80000023404602F0D4FB5AB0BDE8F08100BF18
:100F9000AFF3008026417272DF25D7B700460020EC
:100FA000F0B5254E4FF48A7505FB0065F1B096F853
:100FB000D83085F8DC300024D822214685F8E84076
:100FC0003AA800F0FBFD06F1090000F0EFFDD5F8AE
:100FD000E4308DF8F000C2B206AF06F109010DF160
:100FE000F100CDE93A3400F0C3FD394601223AA8B8
:100FF00001F00EF880B2CDE9047008230127CDE995
:10100000023706F1D803019330230093317A0B485D
:1010100007A3D3E9002302F08BFBA04206DD01F019
:10102000BFFFC5F8E000384671B0F0BD2046FBE7D1
:1010300078F6339F93CACD8D0046002000350020FE
:101040002DE9F0411D4D1E4E1E4F86B0284602F080
:101050009BFB034658B30024CDE90344ADF814408C
:10106000027B8DF8142099684068029403AA03C299
:101070001B68DFF8548043F00043029301F092FFB5
:10108000821941F10003009402A9384601F054FA94
:10109000A04205DD284602F07BFB88F80040D5E73A
:1010A00098F80030072B05D8013388F8003006B0D7
:1010B000BDE8F081014802F06BFBF8E70035002045
:1010C00040420F0030350020354B002070B50D46F2
:1010D00014461E4602F088FA50B9022E10D1012C97
:1010E0000ED112A3D3E90023C5E90023012007E0B4
:1010F000282C10D005D8012C09D0052C0FD00020A9
:1011000070BD302CFBD10BA3D3E90023ECE70BA37C
:10111000D3E90023E8E70BA3D3E90023E4E70BA31B
:10112000D3E90023E0E700BFAFF30080401DA1201A
:1011300026812A0B78F6339F93CACD8D9E6AC421EF
:10114000818A46EE26417272DF25D7B7F017304A02
:1011500039059E5638B505460E4C0021013500F084
:1011600067FCA4F82C55B4F82C0500F049FC78B1C4
:10117000B4F82C0500F054FC014648B9B4F82C052D
:1011800000F056FCB4F82C350133A4F82C35EAE70E
:1011900038BD00BF0046002010B50A4B0A4A1A604D
:1011A00003F5805393F860203AB9DC6D2CB12046EA
:1011B00001F05AF8204605F0EDFDBDE81040034867
:1011C00001F052B830350020E06F0008784500206B
:1011D0002DE9F04F8FB000AF05460C4602F004FA3F
:1011E000002849D1237E022B1BD1E38A012B18D181
:1011F00001F0D6FE0646FFF7E1FD03464FF4C87046
:10120000DFF8C482B3FBF0F206F5167602FB10336A
:1012100016FA83F3C8F80030E37E33B9A34B0022FB
:101220001A703C37BD46BDE8F08F07F12401204617
:1012300000F044FE0028F4D107F11400FFF7D6FDBA
:1012400097F8264007F11401224607F1270005F020
:10125000EBFD0028E2D10F2C08D8944B1C70D8F875
:101260000030A3F51673C8F80030DAE797F82410B9
:10127000284602F0B1F9D4E7E38A282B2BD010D806
:10128000012B23D0052BCCD1BFF34F8F8849894B3D
:10129000CA6802F4E0621343CB60BFF34F8F00BF14
:1012A000FDE7302BBDD1844EE17E327A9142B8D138
:1012B000607E3146002291F8DC50854200F0A58026
:1012C0000132042A01F58A71F5D1AAE721462846A0
:1012D000FFF79CFDA5E721462846FFF703FEA0E7A0
:1012E000B2F8EC507B6005F103094FEA99094FEA27
:1012F0008902D11DC908A8EBC1039D46EB46002118
:10130000584600F05BFC04F1EE012A463144584691
:1013100000F02EFC7B6813B9012000F061FB96F809
:10132000D20000F06DFB044630B9307200F0A0FB33
:10133000204600F055FBB1E0D6F8D4203AB996F833
:10134000D200B6F82C25824201D8FFF703FFD6F869
:10135000D4202A44944208D296F8D200B6F82C251C
:101360000130824201D8FFF7F5FE70685FFA89F21A
:10137000594600F02BFC08B9C54679E0726896F82A
:10138000D2002A447260D6F8D42005EB0209C6F8D0
:10139000D49000F035FB814509D396F8D220D6F8D9
:1013A000D4000132001B86F8D220C6F8D400FF2DED
:1013B0000FD80024347200F05BFB204600F010FBD5
:1013C00000F0D4FE3D4B188108B9FFF70DFAC54671
:1013D00027E7BB6896F8D9000AFB0362FB68D2F8DE
:1013E000E41082F8E83001F58061C2F8E030C2F81C
:1013F000E410FFF7D5FDFFF723FE96F8D920013260
:1014000002F0030286F8D920B6E74FF48A7A0AFB85
:1014100002F505F1EA013144204600F025FEF860AE
:1014200000287FF4FEAE3544012285F8E82001F063
:10143000B7FDD5F8E020D6ED007ADFED216A801AFD
:10144000192838BF192040F6B832904228BF1046FC
:10145000B8EE677A07EE900AF8EEE77A67EEA67ABA
:10146000DFED186AE7EE267AFCEEE77AC6ED007A41
:1014700096F8D930BB60BA6873680AFB02F4321977
:1014800092F8E81059B1D2F8E4108B42E8463FF4E4
:1014900027AF002182F8E810C2F8E010C546736853
:1014A000064A9B0A01331381BBE600BFF9340020D2
:1014B00000ED00E00400FA0500460020E8240020CA
:1014C000CDCCCC3D6666663FFC340020014B1870E5
:1014D000704700BFF424002030B54FF000542B4B70
:1014E00022689A4285B007D004F0DCFA044620BB9B
:1014F0000024204605B030BD254B627D25481A707A
:10150000237D03724FF48073C0F8F8314FF40073F9
:10151000C0F80C3300254FF44073C0F820341E4946
:10152000C0F8E450C922093000F022FB2046E02236
:10153000294600F043FB0124DBE7184A184D136CE1
:1015400043F000731364AA6D164B9A42D0D12B6EF0
:10155000013B7E2BCCD8144A07CA01AB83E80700B5
:101560001846032100F0D0FD6B6D83424FF000035D
:10157000BED12A6D8A4201BFAB65054B2A6E1A7037
:1015800003BF0A4BEA6D1A601C46B2E79AAD44C528
:10159000F4240020004600201600002000380240FD
:1015A000006600405041A0B0586600401023002063
:1015B00037B51A4D00F0DAFD02236B71184B288104
:1015C00019681848012201F089FB00230193164B8A
:1015D000164900931648174B4FF4805201F0D4FF80
:1015E000154B197811B1124801F0F6FF01F0D8FC43
:1015F0000446FFF7E3FB4FF4C873B0FBF3F202FBC2
:10160000130304F5167010FA83F00C4B186004F005
:101610003FFA08B10F232B8103B030BDE82400202E
:101620001023002030350020CD100008F8240020C1
:1016300000350020D1110008F4240020FC340020E3
:101640002DE9F04F2DED028B0FF23829D9E90089F1
:10165000834C93B00BAE9FED7E8BFFF7F1FC814F77
:10166000DFF828A200230A93ADF834300B9373609F
:101670004FF0000B5B468DED008B01250DF11D0237
:1016800007A938468DF81C508DF81DB001F0D6FA28
:101690009DF81C30002B40F0A580204601F0A4FFEF
:1016A0000646002845D1704F01F07AFC3B6898420D
:1016B0003FD301F075FC8246FFF780FB4FF4C873FF
:1016C000B0FBF3F202FB13030AF5167010FA83F075
:1016D0003860664F97F800B0CBF1100ABBF1000FED
:1016E00014BF33462B465FFA8AFA0EA88DF82830CD
:1016F000FFF77CFBBAF1060F28BF4FF0060A0EABCE
:1017000003EB0B0152460DF1290000F031FA0AAB50
:101710000393182302930AF10102554BD2B2CDE98B
:101720000053049220464CA3D3E9002301F0A2FF0A
:101730003E7001F035FC4F4A4F4D1368C31AB3F5A4
:101740007A7F2ED3106001F02DFC02460B46204616
:1017500002F028F8204601F047FF10B32B7A474EDD
:10176000002B14BF03230223737101F019FC0EAF89
:101770004FF47A730122B0FBF3F039463060304603
:1017800000F074FB182302933D4B019380B240F2AA
:101790005513CDE90370009342464B46204601F0B5
:1017A00069FF2B7A93B101F0FBFB002607464FF44B
:1017B0008A7A95F8D900304400F003000AFB005300
:1017C00093F8E82092B30136042EF2D1C82003F03A
:1017D00067FC2B7A002B7FF43DAF13B0BDEC028B7E
:1017E000BDE8F08FDAF8143083F00203CAF8143041
:1017F000594610220EA800F0E1F90DF11E0308AAC7
:101800000AA9384600F096FF96E803000FAB83E87C
:1018100003009DF834308DF844300A9B0E930EA9D6
:10182000DDE90823204602F091F921E7D3F8E02012
:1018300042B12B68FA2B38BFFA23BA1A0533B2EB40
:10184000430FC0D3FFF7ACFB0028BCD1BEE700BFFD
:101850000000000000000000401DA12026812A0B8E
:101860000035002030350020FC340020F934002001
:10187000F8340020304B002000460020E8240020EF
:10188000344B0020F1C6A7C1D068080F0004024005
:1018900008B5054800F0E8FFBDE80840034A0449E0
:1018A000002005F071BA00BF30350020844B0020C5
:1018B00099110008704700002DE9F84F4FF47A7332
:1018C000DFF85880DFF8589006460D4602FB03F714
:1018D000002498F900305A1C5FFA84FA01D0A34220
:1018E00012D159F8240003682A46D3F820B03146B3
:1018F0003B46D847854207D1074B012083F800A01B
:10190000BDE8F88F0124E4E7002CFBD04FF4FA7017
:1019100003F0C6FB0020F3E7784B00201C230020D7
:101920002023002070B504464FF47A76412C2546DA
:1019300028BF412506FB05F003F0B2FB641BF5D17F
:1019400070BD000007B50023024601210DF107001C
:101950008DF80730FFF7B0FF20B19DF8070003B006
:101960005DF804FB4FF0FF30F9E700000A4608B5C8
:101970000421FFF7A1FF80F00100C0B2404208BD82
:1019800030B4074B0A461978064B53F821402368B8
:10199000DD69054B0146AC46204630BC604700BFC0
:1019A000784B002020230020A086010070B503F0B2
:1019B00099FE094E094D30800024286833888342FF
:1019C00008D903F089FE2B6804440133B4F5803F45
:1019D0002B60F2D370BD00BF7A4B0020384B002043
:1019E00003F036BF00F1006000F5803000687047FA
:1019F00000F10060920000F5803003F0C1BE0000ED
:101A0000054B1A68054B1B889B1A834202D9104468
:101A100003F062BE00207047384B00207A4B002054
:101A2000024B1B68184403F05FBE00BF384B002018
:101A3000024B1B68184403F06FBE00BF384B0020F8
:101A400010F003030AD1B0F5047F05D200F1005075
:101A5000A0F51040D0F80038184670470023FBE787
:101A600000F10050A0F51040D0F8100A70470000B7
:101A7000064991F8243033B10023086A81F82430F4
:101A80000822FFF7B5BF0120704700BF3C4B002084
:101A9000014B1868704700BF002004E070B5194B77
:101AA0001D68194B0138C5F30B0408442D0C0422A2
:101AB0001E88A6420BD15C680A46013C824213464E
:101AC0000FD214F9016F4EB102F8016BF6E7013A3B
:101AD00003F10803ECD181420B4602D22C2203F819
:101AE000012B0A4A05241688AE4204D1984284BFCD
:101AF000967803F8016B013C02F10402F3D1581A05
:101B000070BD00BF002004E0846F0008706F000803
:101B1000022802D1044B98617047012802BF024B92
:101B200008229A61704700BF00040240022804D1D5
:101B3000054B4FF400329A6170470128FCD1024BEB
:101B40004FF40022F7E700BF00040240022805D14D
:101B5000064A536983F00203536170470128FCD1A0
:101B6000024A536983F00803F6E700BF000402400D
:101B700010B50023934203D0CC5CC4540133F9E781
:101B800010BD000010B5013810F9013F3BB191F9CB
:101B900000409C4203D11AB10131013AF4E71AB175
:101BA00091F90020981A10BD1046FCE70346024642
:101BB000D01A12F9011B0029FAD1704702440346DA
:101BC000934202D003F8011BFAE770472DE9F8436E
:101BD0001F4D144695F824200746884652BBDFF86F
:101BE00070909CB395F824302BB92022FF214846F1
:101BF0002F62FFF7E3FF95F82400C0F10802A2422C
:101C000028BF2246D6B24146920005EB8000FFF77E
:101C1000AFFF95F82430A41B1E44F6B2082E1744DB
:101C20009044E4B285F82460DBD1FFF721FF00285F
:101C3000D7D108E02B6A03EB82038342CFD0FFF7B2
:101C400017FF0028CBD10020BDE8F8830120FBE777
:101C50003C4B0020024B1A78024B1A70704700BFB1
:101C6000784B00201C23002038B5174C174D204618
:101C700002F046FD2946204602F06EFD2D686A6D91
:101C8000936B23F4002393634FF47A70FFF74AFEBB
:101C90000F49284602F066FE6A6D0E4D936B286868
:101CA0000D4943F400239363A0424FF4E1330B60EA
:101CB00001D002F085FC6868A04204D0BDE838403D
:101CC000054902F07DBC38BD68500020087100084D
:101CD0001071000820230020644B002070B50C4BCD
:101CE0000C4D1E780C4B55F826209A4204460DD018
:101CF0000A4B002114221846FFF760FF04600146DA
:101D000055F82600BDE8704002F05ABC70BD00BF17
:101D1000784B00202023002068500020644B0020D6
:101D20002DE9F0470D46044600219046284640F232
:101D30007912FFF743FF234620220021284601F0B5
:101D4000A7FE231D02222021284601F0A1FE631DCB
:101D500003222221284601F09BFEA31D03222521F8
:101D6000284601F095FE04F1080310222821284698
:101D700001F08EFE04F1100308223821284601F0FC
:101D800087FE04F1110308224021284601F080FE5D
:101D900004F1120308224821284601F079FE04F1DB
:101DA000140320225021284601F072FE04F118038A
:101DB00040227021284601F06BFE04F12003082226
:101DC000B021284601F064FE04F121030822B82165
:101DD000284601F05DFE04F12207C0263B4631464D
:101DE00008222846083601F053FEB6F5A07F07F119
:101DF0000107F3D104F1320308223146284601F0ED
:101E000047FE002704F1330A94F832304FEAC7093D
:101E10009F4209F5A47615D3B8F1000F08D13146D9
:101E200004F599730722284601F032FE09F24F1695
:101E3000274694F832213B1B93420CD3F01DC00877
:101E4000BDE8F0870AEB070308223146284601F077
:101E50001FFE0137D8E707F2331331460822284620
:101E600001F016FE08360137E3E7000013B504461B
:101E70000846002101602346C0F80310202201908B
:101E800001F006FE0198231D0222202101F000FE30
:101E90000198631D0322222101F0FAFD0198A31D80
:101EA0000322252101F0F4FD019804F1080310221A
:101EB000282101F0EDFD072002B010BDF7B5002389
:101EC000047F00910E4607221946054601F0A4FC46
:101ED000731C0093012200230721284601F09CFC7B
:101EE000C4B9B31C0093052223460821284601F0FB
:101EF00093FC0D243746B278BB1B934211D32B7F42
:101F0000A88A0734E408BBB9844294BF00200120AA
:101F100003B0F0BDAB8ADB00083BDB08B3700824DC
:101F2000E8E7FB1C0093214600230822284601F025
:101F300073FC08340137DEE7201A18BF0120E7E7F9
:101F4000F7B50023047F00910E4608221946054686
:101F500001F062FC731CC4B90822009311462346A9
:101F6000284601F059FC1024012372785F1C013BC4
:101F7000934211D32B7FA88A0734E408BBB984426B
:101F800094BF0020012003B0F0BDAB8ADB00083B0A
:101F9000DB0873700824E7E7F31900932146002358
:101FA0000822284601F038FC08343B46DDE7201AB9
:101FB00018BF0120E7E70000F8B50E4605461446B5
:101FC000002181223046FFF7F9FD2B46082200212F
:101FD000304601F05DFD7CB96B1C072208213046BC
:101FE00001F056FD0F2401236A785F1C013B9342E8
:101FF00004D3E01DC008F8BD0824F4E7EB1921461E
:102000000822304601F044FD08343B46ECE700006E
:10201000F8B50E46054614460021CE223046FFF79D
:10202000CDFD2B4628220021304601F031FD7CB940
:1020300005F1080308222821304601F029FD30244B
:102040002F462A7A7B1B934204D3E01DC008F8BDBB
:102050002824F5E707F1090321460822304601F05C
:1020600017FD08340137ECE7F7B5047F00910E4601
:10207000012310220021054601F0CEFBC4B9B31C98
:102080000093092223461021284601F0C5FB19249C
:1020900037467288BB1B9A4211D82B7FA88A073417
:1020A000E408BBB9844294BF0020012003B0F0BD16
:1020B000AB8ADB00103BDB0873801024E8E73B1D94
:1020C0000093214600230822284601F0A5FB08348E
:1020D0000137DEE7201A18BF0120E7E730B5094DC8
:1020E0000A4491420DD011F8013B5840082340F3B7
:1020F0000004013B2C4013F0FF0384EA5000F6D1AA
:10210000EFE730BD2083B8EDF7B54FF0FF33DFF8D0
:1021100054C0DFF854E000EB81011A4688421CD01D
:1021200050F8044B019401AF042417F8015B82EAD4
:1021300005620825DB18164605F1FF355241002ED1
:10214000BCBF83EA0C0382EA0E0215F0FF05F1D151
:10215000013C14F0FF04E8D1E0E7D843D14303B0D9
:10216000F0BD00BF9336EAA9EBE1F042F7B5384A7B
:10217000106851686B4603C36A46364936480823DF
:1021800004F062FE0446002833D10A25334A106861
:1021900051686B4603C36A4631492F48082304F04F
:1021A00053FE0446002849D00369B3F5F81F45D80B
:1021B000B0F8661040F27A5291423FD1294A024467
:1021C00002F15C018B4239D35C3B234900209E1A0B
:1021D000FFF784FF3246074604F164010020FFF751
:1021E0007DFFA3689F4229D1E368984208BF00257C
:1021F00024E00369B3F5F81F27D8418B40F27A52E7
:10220000914220D1174A024402F110018B4218D3A7
:10221000103B114900209D1AFFF760FF2A46064631
:1022200004F118010020FFF759FFA3689E4202D174
:10223000E368984201D00D25A8E70025284603B0A1
:10224000F0BD1025A2E70C25A0E70B259EE700BFF7
:10225000A46F0008DCFF1E0000000108AD6F00083D
:1022600090FF1E000800FFF710B5037C044613B969
:10227000006804F0D1FD204610BD00000023BFF32C
:102280005B8FC360BFF35B8FBFF35B8F8360BFF374
:102290005B8F7047BFF35B8F0068BFF35B8F704746
:1022A00070B505460C30FFF7F5FF05F1080604464A
:1022B0003046FFF7EFFFA04206D930466D68FFF7C2
:1022C000E9FF2544281A70BD3046FFF7E3FF201AC6
:1022D000F9E7000070B50546406898B105F10800BF
:1022E000FFF7D8FF05F10C0604463046FFF7D2FF92
:1022F0008442304694BF6D680025FFF7CBFF013C58
:102300002C44201A70BD000038B50C460546FFF776
:10231000C7FFA04210D305F10800FFF7BBFF04443C
:102320006868B4FBF0F100FB1144BFF35B8F012040
:10233000AC60BFF35B8F38BD0020FCE72DE9F041B6
:10234000144607460D46FFF7C5FF844228BF0446E2
:10235000D4B1B84658F80C6B4046FFF79BFF3044A9
:10236000286040467E68FFF795FF331A9C4203D8E9
:102370006C600120BDE8F0816B60A41B3B68AB6022
:102380002044E8600220F5E72046F3E738B50C4624
:102390000546FFF79FFFA04210D305F10C00FFF7A1
:1023A00079FF04446868B4FBF0F100FB1144BFF30B
:1023B0005B8F0120EC60BFF35B8F38BD0020FCE732
:1023C0002DE9FF41884669460746FFF7B7FF6C468F
:1023D00006B204EBC6060025B44209D06268206844
:1023E00008EB0501FFF7C4FB636808341D44F3E7FD
:1023F00029463846FFF7CAFF284604B0BDE8F081F9
:10240000F8B505460C300F46FFF744FF05F1080606
:1024100004463046FFF73EFFA042304688BF6C6856
:10242000FFF738FF201A386020B130462C68FFF7DC
:1024300031FF2044F8BD000073B5144606460D4632
:10244000FFF72EFF844228BF04460190DCB101A9AA
:102450003046FFF7D5FF019B33B93268C5E9023337
:10246000C5E9002401200CE09C4238BF019428609B
:10247000019868608442F5D93368AB60241AEC6037
:10248000022002B070BD2046FBE700002DE9FF41AD
:102490000F466946FFF7D0FF6C4600B204EBC0055B
:1024A0000026AC4209D0D4F8048054F8081BB819AF
:1024B0004246FFF75DFB4644F3E7304604B0BDE813
:1024C000F081000038B50546FFF7E0FF04460146FD
:1024D0002846FFF719FF204638BD0000302383F35C
:1024E000118862B670470000002383F3118862B63A
:1024F0007047000010B4026854681A4623465DF81D
:10250000044B184701207047002070470020704797
:1025100070470000002070470E20704700F5805083
:1025200090F8C800C0F340007047000000F58050EC
:1025300090F9C90070470000F7B50C68BDF820702D
:1025400014F000541E466FD10B7B082B6CD8FFF79C
:10255000C5FF4569AB685B010CD4AB681B0108D4AF
:10256000AC6814F080545DD1FFF7BEFF204603B085
:10257000F0BD01240B6804F1180C002BB8BFDB0080
:102580004FEA0C1CB4BF43F004035B0545F80C3064
:102590000B680FFA84FC13F0804F18BF05EB0C1E7C
:1025A00005EB0C1C1EBFDEF8803143F00203CEF8B1
:1025B00080310B7BCCF8843105EB04158B68C5F8B2
:1025C0008C314B68C5F88831DCF8803143F0010369
:1025D000CCF8803100EB441541F268031D4403EB55
:1025E00044130344C5E9002608330D4601F10C0CE1
:1025F00055F804EB43F804EB6545F9D184342D8894
:102600001D8000EB441407F00303257925F00B052A
:102610002B432371FFF768FF0097334600F0E2FC7D
:102620000120A4E70224A5E74FF0FF309FE7000058
:1026300013B500F580540191E06DFFF74BFE1F28A4
:102640000AD90199E06D2022FFF7BAFEA0F120031C
:102650005842584102B010BD0020FBE708B500F514
:102660008050FFF73BFFC06DFFF708FEBDE8084054
:10267000FFF73ABF002202608281426082607047A9
:1026800010B500220023C0E9002300230446038183
:102690000C30FFF7EFFF204610BD0000F0B50546F7
:1026A00000F580500C4690F8C83013F0040FC3F3C7
:1026B000800108BF114661F3820304F1840680F8AB
:1026C000C83005EB461389B01B79D8072ED57AB3ED
:1026D00019072DD46846FFF7D3FF05EB441303F524
:1026E000835303F1180703AA103318685968144676
:1026F00003C40833BB422246F7D1186820609B8888
:10270000A380DDE90E23CDE900230123ADF80830D5
:102710002B686946DB6B2846984705EB46152B79F5
:102720001A075CBF43F008032B7101E0002AF4D1C3
:1027300009B0F0BD2DE9F047074688B007F5805491
:1027400068469A468846FFF7C9FE9146FFF798FF0C
:10275000E06DFFF7A5FD1F2829D9E06D202269460D
:10276000FFF7B0FE202822D103AD444605AB2E462C
:1027700003CE9E4220606160354604F10804F6D124
:1027800030682060B388A380DDE90023C9E9002315
:10279000BDF80830AAF80030FFF7A6FE4A465346B7
:1027A0004146384608B0BDE8F04700F009BCFFF7E5
:1027B0009BFE002008B0BDE8F08700002DE9F84F2F
:1027C0000023C0E90133254B044640F8183B0F466F
:1027D000FFF750FF04F12800FFF752FF04F148080B
:1027E00004F582554646083530462036FFF748FF47
:1027F000AE42F9D104F580554FF480534FF00009F3
:10280000C5E91339C5F848800123EE6504F58758FA
:1028100004F58456C5F8549085F8583085F8603032
:10282000083608F108084FF0000A4FF0000B46E99F
:1028300008ABA6F11800FFF71DFF203646F8289CCC
:102840004645F4D185F8C97017B1054800F0A2FBE0
:10285000044B63612046BDE8F88F00BFE06F0008BD
:10286000B86F00080064004010B5044B19780446A6
:102870004A1C1A70FFF7A2FF204610BD804B0020B3
:102880002DE9F047002950D0294B2A4FB7FBF1F52D
:1028900099428CBF0A231123581EB5FBF3FC03FB9E
:1028A0001C53C4B22BB102280346F5D80020BDE862
:1028B000F0870CF1FF36B6F5806FF7D2C4EBC40E8B
:1028C0000EF103034FEAE309C3F3C703A4EB0308C4
:1028D00009F1010A4FF47A755FFA88F009FB055592
:1028E0005AFA88F8B5FBF8F5B5F5617FC1BF0EF16E
:1028F000FF33C3F3C703E01AC0B25C1C50FA84F480
:102900000CFB04F4B7FBF4F4A142CFD1013BDBB2E2
:102910000F2BCBD80138C0B20728C7D800211071BF
:1029200016809170D3700120C1E70846BFE700BF51
:102930003F420F0080DE800270B505460E464FF420
:102940007A746B695B6803F00103B34207D04FF4FC
:102950007A7002F0A5FB013CF3D1204670BD012046
:10296000FCE7000030B54269936913F0700F16D090
:1029700000230B4C936103F1840200EB42121179A6
:102980004D0709D5890707D5416954F823508D6053
:10299000117941F0040111710133032BEBD130BDEA
:1029A000CC6F000873B51D46436916469A68D20776
:1029B000044609D59A6801219960C2F34002CDE925
:1029C00000650021FFF76AFE63699A68D1050BD59F
:1029D0009A684FF480719960C2F34022CDE9006596
:1029E00001212046FFF75AFE63699A68D2030BD58E
:1029F0009A684FF480319960C2F34042CDE9006596
:102A000002212046FFF74AFE204602B0BDE8704092
:102A1000FFF7A8BFF8B50446466900296CD106F156
:102A20000C07386880076AD006EB01153868D5F8BE
:102A3000B00110F0040FD5F8B0011ABFC00840F083
:102A40000040400DA061D5F8B0C11CF0020F1CBFC2
:102A500040F08040A061D5F8B40106EB011100F010
:102A60000F0084F82400D1F8B8012077D1F8B8011C
:102A7000000A6077D1F8B801000CA077D1F8B8014E
:102A8000000EE077D1F8BC0184F82000D1F8BC0139
:102A9000000A84F82100D1F8BC01000C84F822005F
:102AA000D1F8BC11090E84F823103821396004F1E3
:102AB000340004F1180104F1240551F8046B40F8C6
:102AC000046BA942F9D109880180C4E90A2321468F
:102AD0000023238651F8283B2046DB6B984704F5FA
:102AE0008052204692F8C83043F0040382F8C83080
:102AF000BDE8F840FFF736BF06F1100791E7F8BDD3
:102B000010B5044600F04EFA02460B4652EA0301A5
:102B100002D0013A63F100030449086820B121465C
:102B2000BDE81040FFF776BF10BD00BF7C4B002012
:102B3000F8B500F583511E46FFF7D0FCDFF844C01E
:102B40000831002404F1840500EB45152B795F075B
:102B50000ED4DB060CD5D1E900739742B34107D2FE
:102B600043695CF824709F602B7943F004032B7158
:102B70000134032C01F12001E4D1BDE8F840FFF756
:102B8000B3BC00BFCC6F000808B5FFF7A7FCFFF788
:102B9000E9FEBDE80840FFF7A7BC0000F8B54369AF
:102BA0000546986800F0E050B0F1E05F0F461FD096
:102BB000E8B1FFF793FC05F583541034002606F1C5
:102BC000840305EB43131B791A0706D50136032E40
:102BD00004F12004F3D1012007E05B07F6D421467D
:102BE000384600F039FA0028F0D1FFF77DFCF8BD37
:102BF0000120FCE700F5805008B5FFF76FFCC06DC1
:102C0000FFF74EFBFFF770FC43090CBF01200020CB
:102C100008BD0000F8B51D46002313700F46064698
:102C20001446FFF7E7FF80F00100387025B1294610
:102C30003046FFF7B3FF2070F8BD00002DE9B84122
:102C40000C4615461F46804600F0ACF90B4621782D
:102C5000024609B9287850B14046FFF769FFFFF7EF
:102C600093FF3B462A462146FFF7D4FF0120BDE8EB
:102C7000B881000010B5FFF731FC174B1A6C42F019
:102C800000721A641A6A42F000721A621A6A00F537
:102C9000805422F000721A62FFF726FC94F8C830C4
:102CA000DB0718D4B9B103211320FFF717FC01F09B
:102CB000BBFA0321142001F0B7FA0321152001F01B
:102CC000B3FA94F8C83043F0010384F8C830BDE883
:102CD0001040FFF709BC10BD003802402DE9F04755
:102CE00000F5805588B095F8C930012B0446884618
:102CF00016467FD8804F57F823200AB947F823009B
:102D0000D7F800A0C4F80C802674BAF1000F63D085
:102D100095F8C930012B6FD001212046FFF7AAFF9B
:102D2000FFF7DCFB6269136823F00203136062693A
:102D3000136843F001031360636900275F61012199
:102D40002046FFF7D1FBFFF7F7FD002800F0958044
:102D5000E86DFFF793FA04F58359BA4609F10809BB
:102D6000202200216846FEF729FF02A8FFF782FC17
:102D7000CDF818A06A4609EB07030DF1180E94462A
:102D8000BCE80300F44518605960624603F108038B
:102D9000F5D1DCF80000186020379CF804201A7187
:102DA000602FDDD195F8C8306FF38203002785F8D6
:102DB000C8306A4641462046ADF80070ADF8027052
:102DC0008DF80470FFF75CFD636948BB4FF4004267
:102DD0001A6008B0BDE8F08741F2D00003F0DCFFD4
:102DE000814610B15146FFF7E9FCC7F80090B9F1F0
:102DF000000F8DD10020ECE7386803681B6B984703
:102E00000146002888D13868FFF734FF3868036826
:102E100032465B684146984700287FF47DAFE9E77A
:102E200061221A609DF802309DF803201B061204EF
:102E300002F4702203F040731343BDF80020C2F384
:102E4000090213439DF804201205022E02F4E00249
:102E50000CBF4FF000410021134362690B43D36163
:102E6000636913225A616269136823F001031360D6
:102E700039462046FFF760FD08B96369A6E795F873
:102E8000C93093BB6169D1F8002242F00102C1F858
:102E900000226169D1F8002222F47C5222F00E0255
:102EA000C1F800226169D1F8002242F46062C1F8E1
:102EB00000226269C2F814326269C2F8043262699F
:102EC00041F6FF71C2F80C126269C2F840326269C1
:102ED000C2F8443263690122C3F81C226269D2F845
:102EE000003223F00103C2F8003295F8C83043F0F5
:102EF000020385F8C8306CE77C4B002008B500F071
:102F000051F850EA0103024602D0421E61F100016D
:102F1000044B186810B10B46FFF744FDBDE80840AC
:102F200001F064B87C4B002008B50020FFF7E8FDF5
:102F3000BDE8084001F05AB808B50120FFF7E0FDF0
:102F4000BDE8084001F052B800B59BB0EFF309812D
:102F500068226846FEF70CFEEFF30583014B9B6B7E
:102F6000FEE700BF00ED00E008B5FFF7EDFF000051
:102F700000B59BB0EFF3098168226846FEF7F8FDC3
:102F8000EFF30583014B5B6BFEE700BF00ED00E054
:102F9000FEE700000FB408B5029802F00DF8FEE756
:102FA00002F0ACBC02F084BC13B56C4684E80600A9
:102FB000031D94E8030083E80500012002B010BD62
:102FC00073B58568019155B11B885B0707D4D0E9BB
:102FD00000369B6B9847019AC1B23046A847012042
:102FE00002B070BDF0B5866889B005460C465EB18A
:102FF000BDF838305B070AD4D0E900379B6B98479F
:103000002246C1B23846B047012009B0F0BD0022C7
:103010000023CDE900230023ADF808300A4603ABB6
:1030200001F10806106851681C4603C40832B24218
:103030002346F7D1106820609288A280FFF7B2FF84
:103040000423ADF808302B68CDE90001DB6B69463D
:1030500028469847D8E7000030B503680968DD0FB7
:10306000B5EBD17F23F0604421F060424FEAD1708C
:103070000BD0002BB8BFA40C0029B8BF920C94420F
:1030800002D034BF0120002030BD944205D1C1F3ED
:103090008070C3F380738342F6D194422CBF00202A
:1030A0000120F1E72DE9F041456A15B94162BDE81B
:1030B000F0814B6823F06047C3F38A464FEAD37E22
:1030C000C3F3807816EA230638BF3E46AC462B464B
:1030D0005A68BEEBD27F22F060440AD0002A18DA88
:1030E000A40CB44217D19D420FD10D60DEE7134608
:1030F000EEE7A74207D102F08044C2F38072424556
:103100000BD054B1EFE708D2EDE7CCF800100B601C
:10311000CDE7B44201D0B442E5D81A689C46002AF3
:10312000E5D11960C3E700002DE9F047089D01F0E3
:1031300007044FEAD508224405F0070500EBD1004B
:103140004FF47F49944201D1BDE8F08704F00707AE
:1031500005F0070A57453E4638BF5646C6F10806F1
:10316000111B8E4228BF0E46E10808EBD50E415CCC
:1031700013F80EC0B94029FA06F721FA0AF1FFB296
:103180008CEA010147FA0AF739408CEA010C03F88E
:103190000EC034443544D5E780EA0120082341F2CB
:1031A000210201B24000002980B203F1FF33B8BF11
:1031B000504013F0FF03F4D17047000038B50C46BF
:1031C0008D18A54200D138BD14F8011BFFF7E4FFAC
:1031D000F7E7000042684AB1136843604389818978
:1031E00001339BB29942438138BF838110467047B7
:1031F00070B588B0202204460D4668460021FEF7CF
:10320000DDFC20460495FFF7E5FF024658B16B460A
:10321000054608AE1C4603CCB442286069602346CC
:1032200005F10805F6D1104608B070BD082817D979
:1032300009280CD00A280CD00B280CD00C280CD054
:103240000D280CD00E2814BF4020302070470C20D1
:1032500070471020704714207047182070472020B6
:1032600070470000082817D90C280CD910280CD951
:1032700014280CD918280CD920280CD930288CBF38
:103280000F200E207047092070470A2070470B203E
:1032900070470C2070470D20704700002DE9F8435F
:1032A000078C072F04461ED9D0E9029800254FF657
:1032B000FF73C5F12006A5F1200029FA05F108FAEF
:1032C00006F628FA00F031430143C9B21846FFF769
:1032D00063FF0835402D0346EBD1E1693A46BDE86E
:1032E000F843FFF76BBF4FF6FF70BDE8F8830000AF
:1032F00010B54B6823B9CA8A63F30902CA8210BDAC
:1033000004691A681C600361C38A013BC3824A6076
:10331000EFE700002DE9F84F1D46CB8A0F46C3F3B7
:1033200009010529814692460B4630D00020AAB2F9
:1033300007F11A049EB2042E1FFA80F80FD89045A8
:1033400003F1010306D3FB8A0A4462F30903FB82FB
:1033500001201AE01AF80060E6540130EAE79045CF
:10336000F1D2A1F1050B1C237C68BBFBF3F203FB3C
:1033700012BB1FFA8BF6002C45D14846FFF72AFFF7
:10338000044638B978606FF00200BDE8F88F4FF05E
:103390000008E6E7002606607860ADB24FF0000B4B
:1033A000454510D90AEB0803221D13F8011B91555E
:1033B000B1B208F101081B291FFA88F82BD0454546
:1033C00006F10106F1D8FB8AC3F30902154465F33F
:1033D0000903BCE7013292B21C462368002BF9D1E5
:1033E0006B1F0B441C21B3FBF1F301339BB29A42D8
:1033F000D3D2BBF1000FD0D14846FFF7EBFE20B986
:10340000C4F800B0BFE70122E7E7C0F800B05E46AD
:1034100020600446C1E74545D5D94846FFF7DAFEA6
:1034200008B92060AFE7C0F800B00026206004466D
:10343000B6E700002DE9F04F2DED028B1C4683B05E
:103440005B69019207468846002B00F09A80238C26
:103450002BB1E269002A00F09480072B35D807F1E0
:103460000C00FFF7B7FE054638B96FF00205284695
:1034700003B0BDEC028BBDE8F08F14220021FEF7F3
:103480009DFB228CE16905F10800FEF771FB208CA1
:10349000013080B2FFF7E6FEFFF7C8FE013880B2C8
:1034A0002084013028746369228C1B782A4403F03D
:1034B0001F0363F03F0348F0004113723846696010
:1034C0002946FFF7EFFD0125D1E700F10C034FF08E
:1034D000000908EE103A4FF0800A4E464D4618EEAD
:1034E000100AFFF777FE83460028BED01422002181
:1034F000FEF764FB002E3AD1019BABF808300222A4
:103500000BF1080E1FFA82FC0CF10100BCF1060F52
:10351000218C80B201D88E422BD3FFF7A3FEFFF798
:1035200085FE62691278013802F01F028E4208BFE0
:103530004FF0400A42EA49121BFA80F14AEA020AB5
:10354000013048F0004281F808A08BF81000CBF859
:10355000042059463846FFF7A5FD238C0135B342B8
:103560002DB289F001094FF0000AB8D17FE700229F
:10357000C6E7E169895D0EF802100136B6B2013284
:10358000C0E76FF0010572E7F8B515460E46302228
:10359000002104461F46FEF711FB069B6360B5F54C
:1035A000001F079BA76034BF6A094FF6FF72A36232
:1035B00097B2E66104F1100000239A4206D8002376
:1035C0000360A782E3822383E360F8BD06600133D2
:1035D00030462036F1E7000003781BB94BB2002BD0
:1035E000C8BF01707047000000787047F8B50C46FE
:1035F000C969074611B9238C002B37D1257E1F2DB1
:1036000034D8387828BB228C072A2CD8268A36F062
:1036100003032BD14FF6FF70FFF7D0FD20F0010020
:103620003102400441EA0561400C41EA40254FF671
:10363000FF72234629463846FFF7FCFE002807DDC7
:10364000626913780133DBB21F2B88BF002313702C
:10365000F8BD218A2D0645EA012505432046FFF7DE
:103660001DFE0246E5E76FF00300F1E76FF0010091
:10367000EEE7000070B58AB0044616460021282205
:1036800068461D46FEF79AFABDF83830ADF810309E
:103690000F9B05939DF840308DF81830119B0793D0
:1036A0006946BDF84830ADF820302046CDE90265C6
:1036B000FFF79CFF0AB070BD2DE9F041D3690546C4
:1036C0000C4616460BB9138C5BBB377E1F2F28D8D0
:1036D00095F80080B8F1000F26D03046FFF7DEFDE8
:1036E0003378210241EAC33141EA0801338A41EAD1
:1036F000076141EA03410246334641F08001284612
:10370000FFF798FE00280ADD3378012B07D1726994
:1037100013780133DBB21F2B88BF00231370BDE881
:10372000F0816FF00100FAE76FF00300F7E70000A7
:10373000F0B58BB004460D46174600212822684696
:103740001E46FEF73BFA9DF84C305A1E5342534139
:103750008DF800309DF84030ADF81030119B059386
:103760009DF848308DF81830149B07936A46BDF8D1
:103770005430ADF8203029462046CDE90276FFF7D7
:103780009BFF0BB0F0BD0000406A00B104307047F1
:10379000436A1A68426202691A600361C38A013B84
:1037A000C38270472DE9F041D0F82080194E1446AD
:1037B0001D464146002709B9BDE8F081D1E9022341
:1037C000A21A65EB0303964277EB03031ED2036A4A
:1037D0008B420DD1FFF78CFD036A1B6803620369FE
:1037E0000B60C38A0161016A013BC3828846E2E73C
:1037F000FFF77EFD0B68C8F8003003690B60C38AD1
:103800000161013BC382D8F80010D4E788460968FB
:10381000D1E700BF80841E002DE9F04F8BB00D462C
:10382000DDF8509014469B468046002800F0198130
:10383000B9F1000F00F01581531E3F2B00F21181EA
:10384000012A03D1BBF1000F40F00B810023CDE929
:103850000833B8F81430B5EBC30F4FEAC30703D3EE
:1038600000200BB0BDE8F08F2B199F42D8F80C3028
:103870003ABF7F1BFFB227461BB9D8F81030002B88
:103880007AD0272D4ED8C5F12806B7424FF0000355
:103890002CBFF6B23E4600932946D8F8080008AB84
:1038A0003246FFF741FCA7EB060A35445FFA8AFA75
:1038B000B8F8143003F10053053BDB000493D8F84B
:1038C0000C3003932821039B13B1BAF1000F2CD1C4
:1038D000D8F8100040B1BAF1000F05D0009608AB3F
:1038E0005246691AFFF720FC38B2002FB8D066079D
:1038F0000AD00AAB03EBD401624211F8083C02F093
:103900000702134101F8083C082C3CD9102C40F266
:10391000B580202C40F2B780BBF1000F00F09C80F6
:10392000082334E0BA460026C2E7049BE02B28BFF8
:10393000E02306930B44AB42059314D95A1B03981A
:103940000096924534BF5246D2B2691A08AB043091
:103950000792FFF7E9FB079A1644AAEB020A1544FF
:10396000F6B25FFA8AFA049B069A05999B1A0493A9
:10397000039B1B680393A6E70093D8F8080008ABE5
:103980003A462946AEE7BBF1000F13D00123B4EB52
:10399000C30F6CD0082C12D89DF82030621E23FA79
:1039A00002F2D50706D54FF0FF3202FA04F42343A2
:1039B0008DF820309DF8203089F8003051E7102C28
:1039C00012D8BDF82030621E23FA02F2D10706D5C4
:1039D0004FF0FF3202FA04F42343ADF82030BDF873
:1039E0002030A9F800303CE7202C0FD80899631E3E
:1039F00021FA03F3DA0705D54FF0FF3202FA04F497
:103A00000C430894089BC9F800302AE7402C2BD0BF
:103A1000DDE90865611EC4F12102A4F1210326FA43
:103A200001F105FA02F225FA03F311431943CB071A
:103A300012D50122A4F12003C4F1200102FA03F3FC
:103A400022FA01F1A240524243EA010363EB43032D
:103A500032432B43CDE90823DDE90823C9E90023DC
:103A6000FFE66FF00100FCE66FF00800F9E6082CB5
:103A7000A0D9102CB3D9202CEED8C3E7BBF1000F8E
:103A8000ADD0022383E7BBF1000FBBD004237EE758
:103A900030B5012A144638BF0124402C85B028BF18
:103AA00040240025012ACDE9025518D81B788DF84D
:103AB000083063070AD004AB03EBD405624215F863
:103AC000083C02F00702934005F8083C00910346C9
:103AD0002246002102A8FFF727FB05B030BD082AC7
:103AE000E4D9102A03D81B88ADF80830E1E7202A72
:103AF0008DBFD3E900231B680293CDE90223D8E7E9
:103B000010B5CB681BB98B600B618B8210BD04694B
:103B10001A681C600361C38A013BC382CA60F0E774
:103B200003064CBFC0F3C0300220704708B5024600
:103B3000FFF7F6FF022806D15306C2F30F2001D18A
:103B400000F0030008BDC2F30740FBE72DE9F04F8A
:103B500093B0CDE903230A6804461046FFF7E0FF5F
:103B6000022814BFC2F306260026002A0D4682460C
:103B700080F2F28112F0C04940F0EE81097B002909
:103B800000F0EA81022803D02378B34240F0E781B5
:103B9000C2F304630693104602F07F030593FFF718
:103BA000C5FF059B29444FEA834848EA0A4848EA8A
:103BB0004668CE7800230022CDE90823F309834626
:103BC00048EA0008029367D0059B009302466768A5
:103BD000534608A92046B847002800F0C381276A49
:103BE0004FB9414604F10C00FFF702FB074690B9BC
:103BF0006FF0020054E03B6998450DD03F68002FFC
:103C0000F9D1414604F10C00FFF7F2FA074600280B
:103C1000EED0236A3B60276297F817C006F01F08B2
:103C2000CCF3840CACEB08001FFA80FE0028B8BF70
:103C30000EF12000A8EB0C031FFA83FED7E9022146
:103C4000B8BF00B2002B0793BEBF0EF120031BB21A
:103C5000079352EA010338D0039BDFF824E39A1A52
:103C6000049B4FF0000C63EB010196457CEB0103D4
:103C70002BD36B7B97F81AE0734519D1029B002B6D
:103C800078D0012821DC7868F8B9DFF8F0C29445D3
:103C900070EB010316D337E0276A27B96FF00C00E9
:103CA00013B0BDE8F08F3B699845B5D03F68F4E7A5
:103CB000B24890427CEB010301D30020F0E7029B65
:103CC000002BFAD0079B0F2B17DCFA7DB30002F014
:103CD000030203F07C031343FB7539462046FFF7CC
:103CE00007FB6B7BBB76029B3BB9FB7DC3F3840276
:103CF000013262F38603FB75D0E76A7BBB7E9A4292
:103D0000DBD1029B002B35D0B309022B32D0039BB1
:103D1000BB60049BFB60142200210DA8FDF74EFF41
:103D2000039B0A93049B0B932B1D0C932B7BADF8E9
:103D30003EB0013BDBB2ADF83C30069B8DF8423023
:103D4000059B8DF8433094F82C308DF840A083F01B
:103D500001038DF844308DF84180A3680AA92046FC
:103D60009847FB7DC3F38403013303F01F039B02D9
:103D7000FB82A2E7FB7DC6F34012B2EBD31F40F0FB
:103D8000F480C3F38403434540F0F280029A2B7B16
:103D9000B609002A4DD0F2075DD4032B40F2EB8028
:103DA000039BBB60049BFB602B7BAE1D033BDBB224
:103DB0003246394604F10C00FFF7ACFA00280CDA61
:103DC00039462046FFF794FAFB7DC3F384030133A1
:103DD00003F01F039B02FB820AE7DDE90884AB883E
:103DE0003B834FF6FF73C9F12000A9F1200228FAA6
:103DF00009F104FA00F0014324FA02F211431846D3
:103E0000C9B2FFF7C9F909F10809B9F1400F034632
:103E1000E9D1B8822A7B033AD2B23146FFF7CEF914
:103E2000FB7DB882DA43C2F3C01262F3C713FB759D
:103E300043E786B92E1D013BDBB23246394604F119
:103E40000C00FFF767FA0028BADB2A7BB88A013A30
:103E5000D2B23146E2E7F98AC1F30901013B0429F4
:103E6000DAB25BD8281D002307F11B069A4208D955
:103E700010F801CB06F801C0013101330529DBB28E
:103E8000F4D103990A9104990B91934207F11B0114
:103E90000C9138BF043379680D9134BF55FA83F320
:103EA00000230E93FB8AADF83EB0C3F309031A4416
:103EB000069B8DF84230059B8DF8433094F82C30EA
:103EC000ADF83C2083F001038DF8443000238DF8D9
:103ED00040A08DF841807B602A7BB88A013A291D79
:103EE000FFF76CF93B8BB882834203D1A3680AA920
:103EF0002046984720460AA9FFF702FEFB7DBA8AB2
:103F0000C3F38403013303F01F039B02FB823B8B4B
:103F10009A420CBF00206FF01000C1E67B68002BB6
:103F2000AFD0052001E01C3033461E68002EFAD1C8
:103F3000091A081D2E1D184401EB090CBCF11B0FBA
:103F40005FFA89F39DD89A429BD916F8013B00F895
:103F5000013B09F10109EFE76FF00900A0E66FF0FE
:103F60000A009DE66FF00B009AE66FF00D0097E6F1
:103F70006FF00E0094E66FF00F0091E640420F00E4
:103F800080841E00EFF3098305494A6B22F0010289
:103F90004A63683383F30988002383F311887047E9
:103FA00000EF00E0302080F3118862B60C4B0D4A20
:103FB000D96821F4E0610904090C0A43DA60D3F8F6
:103FC000FC20094942F08072C3F8FC200A6842F0E4
:103FD00001020A602022DA7783F82200704700BFCE
:103FE00000ED00E00003FA05001000E010B53023FA
:103FF00083F311880E4B5B6813F4006314D0F1EE69
:10400000103AEFF30984683C4FF08073E361094B89
:10401000DB6B236684F3098800F08CFF10B1064B3C
:10402000A36110BD054BFBE783F31188F9E700BFDF
:1040300000ED00E000EF00E043060008460600083F
:10404000026843681143016003B1184770470000DC
:10405000024AD36843F0C003D36070470044004075
:1040600010B5054C054A0021204600F087FA044AA5
:10407000044BC4E9972310BD884B00205140000831
:104080000044004080DE8002234A037C002918BFE0
:104090000A46012B30B5C0F868220CD11F4B98425C
:1040A00009D11F4B196C41F400311964196E41F4A8
:1040B000003119661B6EB2F904501468D0F86032F2
:1040C000D0F85C12002D03EB5403B3FBF4F3BEBF36
:1040D00023F0070503F0070343EA450394888B6048
:1040E000D38843F040030B61138943F001034B6114
:1040F00044F4045343F02C03CB6004F4A054002395
:104100000B60B4F5806F0B684B680CBF7F23FF23F7
:1041100080F8643230BD00BF20700008884B00205A
:10412000003802402DE9F041D0F85C62F76833684E
:10413000DA0504469DB20DD5302383F311884FF480
:1041400080610430FFF77CFF6FF4807333600023DD
:1041500083F31188302383F3118804F1040815F0E8
:104160002F033AD183F31188380615D5290613D5C4
:10417000302383F3118804F1380000F07BF9002824
:104180004EDA0821201DFFF75BFF4FF67F733B409F
:10419000F360002383F311887A0616D56B0614D5D5
:1041A000302383F31188D4E913239A420AD1236C74
:1041B00043B127F040073F041021201D3F0CFFF7BB
:1041C0003FFFF760002383F31188D4F86822D36897
:1041D00043B3BDE8F041106918472B0714D015F020
:1041E000080F0CBF00214FF48071E80748BF41F071
:1041F0002001AA0748BF41F040016B0748BF41F0CA
:1042000080014046FFF71CFFAD06736805D594F8A2
:1042100064122046194000F0E1F93568ADB29EE71E
:104220007060B6E7BDE8F08100F1604303F56143DB
:104230000901C9B283F80013012200F01F039A405C
:1042400043099B0003F1604303F56143C3F88021F8
:104250001A607047F8B5154682680669AA420B468F
:10426000816938BF8568761AB54204460BD2184674
:104270002A46FDF77DFCA3692B44A361A3685B1B61
:10428000A3602846F8BD0CD918463246FDF770FCED
:10429000AF1BE1683A463044FDF76AFCE3683B44F3
:1042A000EBE718462A46FDF763FCE368E5E7000004
:1042B00083689342F7B51546044638BF8568D0E950
:1042C0000460361AB5420BD22A46FDF751FC6369E9
:1042D0002B446361A36828465B1BA36003B0F0BD59
:1042E0000DD932460191FDF743FC0199E068AF1BFF
:1042F0003A463144FDF73CFCE3683B44E9E72A4693
:10430000FDF736FCE368E4E710B50A440024C36116
:10431000029B8460C0E90000C0E90511C160026130
:10432000036210BD08B5D0E90532934201D182681D
:1043300082B98268013282605A1C42611970D0E9E8
:1043400004329A4224BFC3684361002100F0C4FED6
:10435000002008BD4FF0FF30FBE7000070B53023B0
:1043600004460E4683F31188A568A5B1A368A26927
:10437000013BA360531CA36115782269934224BFBB
:10438000E368A361E3690BB120469847002383F3F8
:104390001188284607E03146204600F08DFE0028AF
:1043A000E2DA85F3118870BD2DE9F74F04460E4619
:1043B00017469846D0F81C904FF0300A8AF31188BF
:1043C0004FF0000B154665B12A4631462046FFF7EF
:1043D00041FF034660B94146204600F06DFE0028CB
:1043E000F1D0002383F31188781B03B0BDE8F08F70
:1043F000B9F1000F03D001902046C847019B8BF311
:104400001188ED1A1E448AF31188DCE7C0E9051112
:10441000C160C3611144009B8260C0E9000001617A
:1044200003627047F8B504460D461646302383F301
:104430001188A768A7B1A368013BA36063695A1CF0
:1044400062611D70D4E904329A4224BFE36863615B
:10445000E3690BB120469847002080F3118807E0FC
:104460003146204600F028FE0028E2DA87F3118862
:10447000F8BD0000D0E905239A4210B501D1826849
:104480007AB98268013282605A1C82611C780369A1
:104490009A4224BFC3688361002100F01DFE2046BC
:1044A00010BD4FF0FF30FBE72DE9F74F04460E46F5
:1044B00017469846D0F81C904FF0300A8AF31188BE
:1044C0004FF0000B154665B12A4631462046FFF7EE
:1044D000EFFE034660B94146204600F0EDFD00289E
:1044E000F1D0002383F31188781B03B0BDE8F08F6F
:1044F000B9F1000F03D001902046C847019B8BF310
:104500001188ED1A1E448AF31188DCE702684368BB
:104510001143016003B11847704700001430FFF7E2
:1045200043BF00004FF0FF331430FFF73DBF0000E2
:104530003830FFF7B9BF00004FF0FF333830FFF7D6
:10454000B3BF00001430FFF709BF00004FF0FF3188
:104550001430FFF703BF00003830FFF763BF0000DF
:104560004FF0FF323830FFF75DBF0000012914BF64
:104570006FF0130000207047FFF772BD37B5154686
:104580000E4A026000224260C0E902220122044673
:1045900002740B46009000F15C014FF480721430FD
:1045A000FFF7B2FE00942B464FF4807204F5AE7113
:1045B00004F13800FFF72AFF03B030BD3470000863
:1045C00010B53023044683F31188FFF75DFD022305
:1045D0002374002080F3118810BD000038B5C36932
:1045E00004460D461BB904210844FFF78FFF2946F6
:1045F00004F11400FFF796FE002806DA201D4FF4A0
:104600000061BDE83840FFF781BF38BD02684368EC
:104610001143016003B118477047000013B5446BA4
:10462000D4F894341A681178042915D1217C022910
:1046300012D11979128901238B4013420CD101A99F
:1046400004F14C0001F0DAFFD4F89444019B217985
:104650000246206800F0D0F902B010BD143001F01D
:104660005DBF00004FF0FF33143001F057BF000072
:104670004C3002F02FB800004FF0FF334C3002F006
:1046800029B80000143001F02BBF00004FF0FF31BB
:10469000143001F025BF00004C3001F0FBBF0000DA
:1046A0004FF0FF324C3001F0F5BF000000207047A2
:1046B00010B5D0F894341A6811780429044617D13B
:1046C000017C022914D15979528901238B4013426C
:1046D0000ED1143001F0BEFE024648B1D4F8944425
:1046E0004FF4807361792068BDE8104000F072B922
:1046F00010BD0000406BFFF7DBBF000070470000FB
:104700007FB5124B036000234360C0E902330125EB
:1047100002260F4B057404460290019300F18402B7
:10472000294600964FF48073143001F06FFE094B58
:104730000294CDE9006304F523724FF48073294697
:1047400004F14C0001F036FF04B070BD5C7000084D
:10475000F54600081D4600080B68302282F31188D8
:104760000A7903EB820290614A79093243F8220008
:104770008A7912B103EB820398610223C0F8941482
:104780000374002080F311887047000038B5037F60
:10479000044613B190F85430ABB9201D0125022115
:1047A000FFF734FF04F1140025776FF0010100F0EA
:1047B0009FFC84F8545004F14C006FF00101BDE8F7
:1047C000384000F095BC38BD10B5012104460430D6
:1047D000FFF71CFF0023237784F8543010BD00003E
:1047E00038B504460025143001F028FE04F14C00D1
:1047F000257701F0F7FE201D84F854500121FFF7C2
:1048000005FF2046BDE83840FFF752BF90F844301E
:1048100003F06003202B07D190F84520212A4FF0A8
:10482000000303D81F2A06D800207047222AFBD194
:10483000C0E90E3303E0034A82630722C2630364C4
:10484000012070472823002037B5D0F894341A6827
:104850001178042904461AD1017C022917D119794B
:10486000128901238B40134211D100F14C052846D7
:1048700001F078FF58B101A9284601F0BFFED4F835
:104880009444019B21790246206800F0B5F803B0FA
:1048900030BD0000F0B500EB810385B09E69044691
:1048A0000D46FEB1302383F3118804EB8507301DDC
:1048B0000821FFF7ABFEFB685B691B6806F14C0043
:1048C0001BB1019001F0A8FE019803A901F096FE2A
:1048D000024648B1039B2946204600F08DF800238C
:1048E00083F3118805B0F0BDFB685A691268002A8D
:1048F000F5D01B8A013B1340F1D104F14402EAE7F1
:10490000093138B550F82140DCB1302383F31188E8
:10491000D4F894241368527903EB8203DB689B6913
:104920005D6845B104216018FFF770FE294604F167
:10493000140001F099FD2046FFF7BAFE002383F32F
:10494000118838BD7047000001F00EB901230370D3
:104950000023C0E90133C36183620362C36243621F
:104960000363704738B50446302383F3118800256C
:10497000C0E90355C0E90555416001F005F902237E
:10498000237085F31188284638BD000070B500EB10
:10499000810305465069DA600E46144618B11022AC
:1049A0000021FDF70BF9A06918B110220021FDF7D5
:1049B00005F931462846BDE8704001F0AFB9000066
:1049C000826802F0011282600022C0E90422826142
:1049D00001F030BAF0B400EB81044789E4680125A6
:1049E000A4698D403D43458123600023A26063603C
:1049F000F0BC01F04BBA0000F0B400EB8104078971
:104A0000E468012564698D403D43058123600023EE
:104A1000A2606360F0BC01F0C5BA000070B502236B
:104A2000002504460370C0E90255C0E90455C56479
:104A3000856180F8345001F00DF963681B6823B17B
:104A400029462046BDE87040184770BD0378052B05
:104A500010B504460AD080F850300523037043682F
:104A60001B680BB1042198470023A36010BD000010
:104A70000178052906D190F85020436802701B6820
:104A800003B118477047000070B590F83430044601
:104A900013B1002380F8343004F14402204601F0C1
:104AA000EBF963689B68B3B994F8443013F0600580
:104AB00035D00021204601F08BFC0021204601F07A
:104AC0007DFC63681B6813B10621204698470623C6
:104AD00084F8343070BD204698470028E4D0B4F8FC
:104AE0004A30E26B9A4288BFE36394F94430E56B45
:104AF000002B4FF0300380F20381002D00F0F28094
:104B0000092284F8342083F311880021D4E90E238C
:104B10002046FFF771FF002383F31188DAE794F84A
:104B2000452003F07F0343EA022340F2023293421E
:104B300000F0C58021D8B3F5807F48D00DD8012B77
:104B40003FD0022B00F09380002BB2D104F14C0235
:104B5000A2630222E2632364C1E7B3F5817F00F020
:104B60009B80B3F5407FA4D194F84630012BA0D1AF
:104B7000B4F84C3043F0020332E0B3F5006F4DD08F
:104B800017D8B3F5A06F31D0A3F5C063012B90D82F
:104B9000636894F846205E6894F84710B4F848308B
:104BA0002046B047002884D04368A3630368E363CA
:104BB0001AE0B3F5106F36D040F6024293427FF40C
:104BC00078AF5C4BA3630223E3630023C3E794F84D
:104BD0004630012B7FF46DAFB4F84C3023F0020364
:104BE000C4E90E55A4F84C30256478E7B4F8443095
:104BF000B3F5A06F0ED194F8463084F84E302046BD
:104C000001F080F863681B6813B1012120469847C2
:104C1000032323700023C4E90E339CE704F14F0300
:104C2000A3630123C3E72378042B10D1302383F33C
:104C300011882046FFF7C4FE85F3118803216368BD
:104C400084F84F5021701B680BB12046984794F8A8
:104C50004630002BDED084F84F3004232370636885
:104C60001B68002BD6D0022120469847D2E794F843
:104C700048301D0603F00F0120460AD501F0EEF87A
:104C8000012804D002287FF414AF2B4B9AE72B4B5A
:104C900098E701F0D5F8F3E794F84630002B7FF45D
:104CA00008AF94F8483013F00F01B3D01A0620462D
:104CB00002D501F0A1FBADE701F094FBAAE794F85F
:104CC0004630002B7FF4F5AE94F8483013F00F0116
:104CD000A0D01B06204602D501F07AFB9AE701F02E
:104CE0006DFB97E7142284F8342083F311882B4658
:104CF0002A4629462046FFF76DFE85F31188E9E62E
:104D00005DB1152284F8342083F311880021D4E9A1
:104D10000E232046FFF75EFEFDE60B2284F83420CA
:104D200083F311882B462A4629462046FFF764FE66
:104D3000E3E700BF8C7000088470000888700008EA
:104D400038B590F834300446002B3ED0063BDAB23A
:104D50000F2A34D80F2B32D8DFE803F0373131086F
:104D6000223231313131313131313737C56BB0F821
:104D70004A309D4214D2C3681B8AB5FBF3F203FB91
:104D800012556DB9302383F311882B462A462946E4
:104D9000FFF732FE85F311880A2384F834300EE0E1
:104DA000142384F83430302383F3118800231A4607
:104DB00019462046FFF70EFE002383F3118838BD05
:104DC000036C03B198470023E7E70021204601F078
:104DD000FFFA0021204601F0F1FA63681B6813B165
:104DE0000621204698470623D7E7000010B590F823
:104DF0003430142B044629D017D8062B05D001D8FF
:104E00001BB110BD093B022BFBD80021204601F04D
:104E1000DFFA0021204601F0D1FA63681B6813B164
:104E2000062120469847062319E0152BE9D10B23CC
:104E300080F83430302383F3118800231A46194652
:104E4000FFF7DAFD002383F31188DAE7C3689B6973
:104E50005B68002BD5D1036C03B19847002384F81D
:104E60003430CEE700230375826803691B689968B4
:104E70009142FBD25A6803604260106058607047EC
:104E800000230375826803691B6899689142FBD807
:104E90005A680360426010605860704708B5084661
:104EA000302383F311880B7D032B05D0042B0DD009
:104EB0002BB983F3118808BD8B6900221A604FF06B
:104EC000FF338361FFF7CEFF0023F2E7D1E9003221
:104ED00013605A60F3E70000FFF7C4BF054BD968C1
:104EE0000875186802681A60536001220275D8605C
:104EF000FBF792BBF84D002030B50C4BDD684B1C26
:104F000087B004460FD02B46094A684600F084F962
:104F10002046FFF7E3FF009B13B1684600F086F9D7
:104F2000A86907B030BDFFF7D9FFF9E7F84D0020B9
:104F30009D4E0008044B1A68DB6890689B68984295
:104F400094BF002001207047F84D0020084B10B599
:104F50001C68D86822681A60536001222275DC60E0
:104F6000FFF78EFF01462046BDE81040FBF754BB1B
:104F7000F84D0020044B1A68DB6892689B689A42DF
:104F800001D9FFF7E3BF7047F84D002038B5074C53
:104F900007490848012300252370656001F01AFCC9
:104FA0000223237085F3118838BD00BF60500020B4
:104FB00094700008F84D002008B572B6044B1865CF
:104FC00000F05AFC00F018FD024B03221A70FEE7B5
:104FD000F84D00206050002000F05EB9EFF3118022
:104FE00020B9EFF30583302282F311887047000067
:104FF00010B530B9EFF30584C4F3080414B180F39D
:10500000118810BDFFF7B6FF84F31188F9E700009F
:10501000034A516853685B1A9842FBD8704700BF37
:10502000001000E08B60022308618B820846704705
:105030008368A3F1840243F8142C026943F8442CDA
:10504000426943F8402C094A43F8242CC26843F8CB
:10505000182C022203F80C2C002203F80B2C044A13
:1050600043F8102CA3F12000704700BF3106000860
:10507000F84D002008B5FFF7DBFFBDE80840FFF75B
:105080002BBF0000024BDB6898610F20FFF726BFA3
:10509000F84D0020302383F31188FFF7F3BF0000A1
:1050A00008B50146302383F311880820FFF724FF59
:1050B000002383F3118808BD064BDB6839B14268D1
:1050C00018605A60136043600420FFF715BF4FF06B
:1050D000FF307047F84D00200368984206D01A68E8
:1050E0000260506099611846FFF7F6BE70470000F5
:1050F00038B504460D462068844200D138BD0368A7
:1051000023605C608561FFF7E7FEF4E710B5036894
:105110009C68A2420CD85C688A600B604C6021607D
:10512000596099688A1A9A604FF0FF33836010BD06
:105130001B68121BECE700000A2938BF0A2170B572
:1051400004460D460A26601901F03EFB01F02AFBD9
:10515000041BA54203D8751C2E460446F3E70A2E0D
:1051600004D9BDE87040012001F074BB70BD00009F
:10517000F8B5144B0D46D96103F1100141600A2ABC
:105180001969826038BF0A22016048601861A81856
:10519000144601F00BFB0A2701F004FB431BA3425A
:1051A000064606D37C1C281901F00EFB274635461F
:1051B000F2E70A2F04D9BDE8F840012001F04ABB0C
:1051C000F8BD00BFF84D0020F8B506460D4601F0C9
:1051D000E9FA0F4A134653F8107F9F4206D12A4638
:1051E00001463046BDE8F840FFF7C2BFD169BB6851
:1051F000441A2C1928BF2C46A34202D92946FFF78E
:105200009BFF224631460348BDE8F840FFF77EBFCA
:10521000F84D0020084E002010B4C0E903230023FD
:105220005DF8044B4361FFF7CFBF000010B5194C88
:10523000236998420DD0D0E90032816813605A602A
:105240009A680A449A60002303604FF0FF33A36119
:1052500010BD2346026843F8102F536000220260FD
:1052600022699A4203D1BDE8104001F0A7BA9368C1
:1052700081680B44936001F095FA2269E1699268B4
:10528000441AA242E4D91144BDE81040091AFFF7BC
:1052900053BF00BFF84D00202DE9F047DFF8BC8078
:1052A00008F110072C4ED8F8105001F07BFAD8F80E
:1052B0001C40AA68031B9A423ED81444D5E9003228
:1052C0004FF00009C8F81C4013605A60C5F8009000
:1052D000D8F81030B34201D101F070FA89F3118887
:1052E000D5E9033128469847302383F311886B6949
:1052F000002BD8D001F056FA6A69A0EB04094A45A0
:1053000082460DD2022001F0A5FA0022D8F8103012
:10531000B34208D151462846BDE8F047FFF728BF01
:10532000121A2244F2E712EB090938BF4A4629460D
:105330003846FFF7EBFEB5E7D8F81030B34208D097
:105340001444211AC8F81C00A960BDE8F047FFF713
:10535000F3BEBDE8F08700BF084E0020F84D0020E6
:1053600000207047FEE70000704700004FF0FF305C
:105370007047000002290CD0032904D001290748F6
:1053800018BF00207047032A05D8054800EBC2006B
:105390007047044870470020704700BF6C710008D8
:1053A000382300202071000870B59AB005460846E1
:1053B00001A9144600F0C2F801A8FCF7F7FB431C52
:1053C0005B00C5E900340022237003236370C6B27A
:1053D00001AB02341046D1B28E4204F1020401D86E
:1053E0001AB070BD13F8011B04F8021C04F8010C7C
:1053F0000132F0E708B5302383F311880348FFF743
:1054000023FA002383F3118808BD00BF68500020F1
:1054100090F8443003F01F02012A07D190F845208C
:105420000B2A03D10023C0E90E3315E003F060031B
:10543000202B08D1B0F848302BB990F84520212A0C
:1054400003D81F2A04D8FFF7E1B9222AEBD0FAE7E4
:10545000034A82630722C26303640120704700BFCE
:105460002F23002007B5052917D8DFE801F019160A
:1054700003191920302383F31188104A0190012168
:10548000FFF784FA01980E4A0221FFF77FFA0D48D0
:10549000FFF7A6F9002383F3118803B05DF804FB3E
:1054A000302383F311880748FFF770F9F2E73023C0
:1054B00083F311880348FFF787F9EBE7C070000812
:1054C000E47000086850002038B50C4D0C4C0D49B4
:1054D0002A4604F10800FFF767FF05F1CA0204F14C
:1054E00010000949FFF760FF05F5CA7204F11800C2
:1054F0000649BDE83840FFF757BF00BF30550020D0
:1055000038230020A0700008AA700008B5700008B9
:1055100070B5044608460D46FCF748FBC6B2204667
:10552000013403780BB9184670BD32462946FCF7A2
:1055300029FB0028F3D10120F6E700002DE9F04710
:1055400005460C46FCF732FB2C49C6B22846FFF74D
:10555000DFFF08B10836F6B229492846FFF7D8FF21
:1055600008B11036F6B2632E0BD8DFF89080DFF862
:105570009090244FDFF898A02E7846B92670BDE8A9
:10558000F08729462046BDE8F04701F0C3BC252E30
:1055900030D1072241462846FCF7F4FA80B91A4B6D
:1055A000224603F10C0153F8040B42F8040B8B4222
:1055B000F9D119889B781180937007350F34DBE798
:1055C000082249462846FCF7DDFA98B90F4BA21C81
:1055D000197809090232C95D02F8041C13F8011B8D
:1055E00001F00F015345C95D02F8031CF0D11834D6
:1055F0000835C1E704F8016B0135BDE78C7100087F
:10560000B570000894710008326F0008107AFF1F0F
:105610001C7AFF1FBFF34F8F024AD368DB03FCD411
:10562000704700BF003C024008B5094B1B7873B9B6
:10563000FFF7F0FF074B1A69002ABFBF064A5A60FE
:1056400002F188325A601A6822F480621A6008BD3A
:105650008E570020003C02402301674508B50B4BE4
:105660001B7893B9FFF7D6FF094B1A6942F0004245
:105670001A611A6842F480521A601A6822F4805241
:105680001A601A6842F480621A6008BD8E570020C2
:10569000003C02401728F0B516D80C4C0C49237872
:1056A0007BB90C4D0E4618234FF0006255F8047B71
:1056B00046F8042B013B13F0FF033A44F6D10123D3
:1056C000237051F82000F0BD0020FCE7F0570020C7
:1056D00090570020A8710008014B53F82000704734
:1056E000A871000818207047172810B5044601D982
:1056F000002010BDFFF7CEFF064B53F824301844AE
:10570000C21A0BB90120F4E712680132F0D1043B50
:10571000F6E700BFA8710008172838B5044628D856
:105720001549FFF777FFFFF77FFFF323CB600C23CB
:10573000B0FBF3F203FB1205D30143EAC503DBB26E
:1057400043F4007343F002030B610B6943F48033AD
:105750000B61FFF75FFFFFF79DFF084B53F8241025
:1057600000F046F9FFF77AFF2046BDE83840FFF722
:10577000BBBF002038BD00BF003C0240A87100083C
:10578000F8B512F00103144642D18218B2F1026F4B
:1057900057D82D4B1B6813F0010352D02B4DFFF748
:1057A00043FFF323EB60FFF735FF40F20127032CA3
:1057B00015D824F001046618244C401A40F2011751
:1057C000B142236900EB010524D123F001032361D9
:1057D000FFF744FF0120F8BD043C0430E7E78307EE
:1057E000E7D12B6923F440732B612B693B432B6179
:1057F00051F8046B0660BFF34F8FFFF70BFF036890
:105800009E42E9D02B6923F001032B61FFF726FFAD
:105810000020E0E723F44073236123693B432361C5
:105820000B882B80BFF34F8FFFF7F4FE2D8831F8E4
:10583000023BADB2AB42C3D0236923F00103236125
:10584000E4E71846C7E700BF00380240003C0240CA
:10585000084908B50B7828B11BB9FFF7E5FE01230D
:105860000B7008BD002BFCD0BDE808400870FFF7A6
:10587000F5BE00BF8E57002008B54FF440314FF001
:10588000005000F0B7F8BDE808404FF480314FF009
:10589000805000F0AFB800000846114601F09EBAF3
:1058A000012001F09BBA0000084601F0B5BA0000E3
:1058B00070B582B0FFF792FB0E4E054600F072FF06
:1058C0003268904237BF0C4A0B49516814682EBFAA
:1058D000D1E90041013151600419034641F1000151
:1058E000284601913360FFF783FB0199204602B0FF
:1058F00070BD00BFF4570020F857002070B582B08B
:10590000FFF76CFB104E054600F04CFF32689042EA
:1059100037BF0E4A0D49516814682EBFD1E90041C6
:1059200001315160041941F10001034628460191FB
:105930003360FFF75DFB01994FF47A720023204634
:10594000FAF756FC02B070BDF4570020F85700205B
:1059500010B50244064BD2B2904200D110BD441C97
:1059600000B253F8200041F8040BE0B2F4E700BFA6
:10597000502800400F4B30B51C6F240407D41C6F17
:1059800044F400741C671C6F44F400441C670A4C08
:10599000236843F4807323600244084BD2B29042E0
:1059A00000D130BD441C00B251F8045B43F82050D4
:1059B000E0B2F4E700380240007000405028004098
:1059C00007B5012201A90020FFF7C2FF019803B02B
:1059D0005DF804FB13B50446FFF7F2FFA04205D0C3
:1059E000012201A900200194FFF7C4FF02B010BDFD
:1059F000704700007047000070470000094B5A884C
:105A0000B2F5805F10460BD022F0020341F2010292
:105A1000934205D041F20703C31A584258417047D8
:105A200001207047002004E0074B45F255521A60F0
:105A300002225A6040F6FF729A604CF6CC421A601D
:105A4000024B01221A7070470030004004580020B9
:105A5000034B1B781BB1034B4AF6AA221A6070470E
:105A60000458002000300040034B1A681AB9034A5A
:105A7000D2F874281A6070470058002000300240A5
:105A8000024B4FF08072C3F8742870470030024018
:105A900008B5FFF7E9FF024B1868C0F3407008BD76
:105AA0000058002008B5FFF7DFFF024B1868C0F36D
:105AB000007008BD0058002070470000FEE700009D
:105AC0000A4B0B480B4A90420BD30B4BDA1C121AB1
:105AD000C11E22F003028B4238BF00220021FCF7D6
:105AE0006DB853F8041B40F8041BECE7047400087D
:105AF00008590020085900200859002070B5D0E945
:105B000015439E6800224FF0FF3504EB421351010C
:105B1000D3F800090028BEBFD3F8000940F0804048
:105B2000C3F80009D3F8000B0028BEBFD3F8000B60
:105B300040F08040C3F8000B013263189642C3F86E
:105B40000859C3F8085BE0D24FF00113C4F81C38C1
:105B500070BD0000890141F02001016103699B06CD
:105B6000FCD41220FFF754BA10B5054C2046FEF7BE
:105B7000EDFE4FF0A0436365024BA36510BD00BF6F
:105B8000085800202C72000870B50378012B0546D8
:105B900050D12A4B446D98421BD1294B5A6B42F08D
:105BA00080025A635A6D42F080025A655A6D5A69F2
:105BB00042F080025A615A6922F080025A610E2135
:105BC00043205B69FEF730FB1E4BE3601E4BC4F8BD
:105BD00000380023C4F8003EC02323606E6D4FF4EC
:105BE0005023A3633369002BFCDA012333610C20BB
:105BF000FFF70EFA3369DB07FCD41220FFF708FA2F
:105C00003369002BFCDA0026A6602846FFF776FFF2
:105C10006B68C4F81068DB68C4F81468C4F81C68C2
:105C20004BB90A4BA3614FF0FF336361A36843F0A4
:105C30000103A36070BD064BF4E700BF08580020C5
:105C4000003802404014004003002002003C30C0F5
:105C5000083C30C0F8B5446D054600212046FFF7EA
:105C600079FFA96D00234FF001128F68C4F8343812
:105C70004FF00066C4F81C284FF0FF3004EB4312CD
:105C800001339F42C2F80069C2F8006BC2F80809EC
:105C9000C2F8080BF2D20B686A6DEB6563621023E1
:105CA0001361166916F01006FBD11220FFF7B0F948
:105CB000D4F8003823F4FE63C4F80038A36943F431
:105CC000402343F01003A3610923C4F81038C4F83B
:105CD00014380A4BEB604FF0C043C4F8103B084B3C
:105CE000C4F8003BC4F81069C4F80039EB6D03F147
:105CF000100243F48013EA65A362F8BD087200083D
:105D000040800010426D90F84E10D2F8003823F415
:105D1000FE6343EA0113C2F8003870472DE9F843E7
:105D200000EB8103456DDA68166806F00306731E02
:105D3000022B05EB41130C4680460FFA81F94FEA1E
:105D400041104FF00001C3F8101B4FF0010104F1A6
:105D5000100398BFB60401FA03F391698EBF334E66
:105D600006F1805606F5004600293AD0578A04F11C
:105D70005801490137436F50D5F81C180B43C5F83B
:105D80001C382B180021C3F8101953690127611E14
:105D9000A7409BB3138A928B9B08012A88BF534369
:105DA000D8F85C20981842EA034301F1400205EB61
:105DB0008202C8F85C00214653602846FFF7CAFEFD
:105DC00008EB8900C3681B8A43EA845348346401A2
:105DD0001E432E51D5F81C381F43C5F81C78BDE86A
:105DE000F88305EB4917D7F8001B21F40041C7F8E9
:105DF000001BD5F81C1821EA0303C0E704F13F0398
:105E000005EB83030A4A5A6028462146FFF7A2FEA3
:105E100005EB4910D0F8003923F40043C0F80039ED
:105E2000D5F81C3823EA0707D7E700BF0080001029
:105E300000040002826D1268C265FFF75FBE0000B9
:105E40005831436D49015B5813F4004004D013F4FA
:105E5000001F0CBF02200120704700004831436D35
:105E600049015B5813F4004004D013F4001F0CBF29
:105E7000022001207047000000EB8101CB68196A05
:105E80000B6813604B6853607047000000EB8103A0
:105E900030B5DD68AA691368D36019B9402B84BF97
:105EA000402313606B8A1468426D1C44013CB4FBB0
:105EB000F3F46343033323F0030302EB411043EA9B
:105EC000C44343F0C043C0F8103B2B6803F0030306
:105ED000012B09B20ED1D2F8083802EB411013F4AD
:105EE000807FD0F8003B14BF43F0805343F0005351
:105EF000C0F8003B02EB4112D2F8003B43F00443F0
:105F0000C2F8003B30BD00002DE9F041244D6E6D1C
:105F100006EB40130446D3F8087BC3F8087B380728
:105F20000AD5D6F81438190706D505EB840321469F
:105F3000DB6828465B689847FA071FD5D6F81438FF
:105F4000DB071BD505EB8403D968CCB98B69488A7C
:105F50005A68B2FBF0F600FB16228AB91868DA68B4
:105F600090420DD2121AC3E90024302383F3118822
:105F70000B482146FFF78AFF84F31188BDE8F081C2
:105F8000012303FA04F26B8923EA02036B81CB68D5
:105F9000002BF3D021460248BDE8F041184700BF6E
:105FA0000858002000EB810370B5DD68436D6C6913
:105FB0002668E6604A0156BB1A444FF40020C2F836
:105FC00010092A6802F00302012A0AB20ED1D3F89E
:105FD000080803EB421410F4807FD4F8000914BFC2
:105FE00040F0805040F00050C4F8000903EB42122A
:105FF000D2F8000940F00440C2F80009D3F8340890
:10600000012202FA01F10143C3F8341870BD19B935
:10601000402E84BF4020206020682E8A8419013CD5
:10602000B4FBF6F440EAC44040F000501A44C6E71E
:106030002DE9F8433B4D6E6D06EB40130446D3F853
:106040000889C3F8088918F0010F4FEA40171AD0E1
:10605000D6F81038DB0716D505EB8003D9684B69F5
:106060001868DA68904230D2121A4FF000091A60AC
:10607000C3F80490302383F3118821462846FFF7A4
:1060800091FF89F3118818F0800F1CD0D6F83438AE
:106090000126A640334216D005EB84036D6DD3F87C
:1060A0000CC0DCF814200134E4B2D2F800E005EBB7
:1060B00004342F445168714515D3D5F8343823EA98
:1060C0000606C5F83468BDE8F883012303FA04F234
:1060D0002B8923EA02032B818B68002BD3D0214626
:1060E00028469847CFE7BCF81000AEEB0103834287
:1060F00028BF0346D7F8180980B2B3EB800FE2D867
:106100009068A0F1040959F8048FC4F80080A0EB4E
:1061100009089844B8F1040FF5D818440B4490606E
:106120005360C7E7085800202DE9F74FA24C656D72
:106130006E69AB691E4016F480586E6107D0204628
:10614000FEF76CFC03B0BDE8F04FFDF74FBF002E2B
:1061500012DAD5F8003E98489B071EBFD5F8003EDE
:1061600023F00303C5F8003ED5F8043823F00103FB
:10617000C5F80438FEF77CFC370505D58E48FFF7D7
:10618000BDFC8D48FEF762FCB0040CD5D5F808388C
:1061900013F0060FEB6823F470530CBF43F4105355
:1061A00043F4A053EB6031071BD56368DB681BB970
:1061B000AB6923F00803AB612378052B0CD1D5F82C
:1061C000003E7D489A071EBFD5F8003E23F003032A
:1061D000C5F8003EFEF74CFC6368DB680BB17648FF
:1061E0009847F30274D4B70227D5D4F85490DFF857
:1061F000C8B100274FF0010A09EB4712D2F8003B63
:1062000003F44023B3F5802F11D1D2F8003B002BCB
:106210000DDA62890AFA07F322EA0303638104EBC9
:106220008703DB68DB6813B1394658469847A36D8E
:1062300001379B68FFB29F42DED9F00617D5676D24
:106240003A6AC2F30A1002F00F0302F4F012B2F538
:10625000802F00F08580B2F5402F08D104EB830336
:106260000022DB681B6A07F5805790426AD1300331
:10627000D5F8184813D5E10302D50020FFF744FEF6
:10628000A20302D50120FFF73FFE630302D50220DF
:10629000FFF73AFE270302D50320FFF735FE75030B
:1062A0007FF550AFE00702D50020FFF7C1FEA10740
:1062B00002D50120FFF7BCFE620702D50220FFF7DE
:1062C000B7FE23077FF53EAF0320FFF7B1FE39E7A6
:1062D000636DDFF8E4A0019300274FF00109A36D7F
:1062E0009B685FFA87FB9B453FF67DAF019B03EB05
:1062F0004B13D3F8001901F44021B1F5802F1FD1C1
:10630000D3F8001900291BDAD3F8001941F09041A5
:10631000C3F80019D3F800190029FBDB5946606D5A
:10632000FFF718FC218909FA0BF321EA0303238103
:1063300004EB8B03DB689B6813B1594650469847C2
:106340000137CCE7910708BFD7F80080072A98BF2C
:1063500003F8018B02F1010298BF4FEA182884E785
:10636000023304EB830207F580575268D2F818C055
:10637000DCF80820DCE9001CA1EB0C0C00218842B1
:106380000AD104EB830463689B699A6802449A60AB
:106390005A6802445A606AE711F0030F08BFD7F841
:1063A00000808C4588BF02F8018B01F1010188BF94
:1063B0004FEA1828E3E700BF08580020436D03EBBD
:1063C0004111D1F8003B43F40013C1F8003B704782
:1063D000436D03EB4111D1F8003943F40013C1F8C8
:1063E00000397047436D03EB4111D1F8003B23F4B2
:1063F0000013C1F8003B7047436D03EB4111D1F826
:10640000003923F40013C1F80039704730B5039CFC
:106410000172043304FB0325C0E90653049B0363A4
:106420000021059BC160C0E90000C0E90422C0E969
:106430000842C0E90A11436330BD0000416A0022EE
:10644000C0E90411C0E90A22C2606FF00101FEF741
:106450004FBE0000D0E90432934201D1C2680AB9AC
:10646000181D70470020704703691960C268013227
:10647000C260C269134482690361934224BF436AC4
:1064800003610021FEF728BE38B504460D46E368D7
:106490003BB16269131D1268A3621344E3620020DA
:1064A00007E0237A33B929462046FEF705FE002887
:1064B000EDDA38BD6FF00100FBE70000C368C26988
:1064C000013BC3604369134482694361934224BF23
:1064D000436A436100238362036B03B1184770472B
:1064E00070B53023044683F31188866A3EB9FFF7FE
:1064F000CBFF054618B186F31188284670BDA36A04
:10650000E26A13F8015BA362934202D32046FFF7CD
:10651000D5FF002383F31188EFE700002DE9F84F42
:1065200004460E46174698464FF0300989F3118805
:106530000025AA46D4F828B0BBF1000F09D1414686
:106540002046FFF7A1FF20B18BF311882846BDE854
:10655000F88FD4E90A12A7EB050B521A934528BF0E
:106560009346BBF1400F1BD9334601F1400251F86D
:10657000040B43F8040B9142F9D1A36A403340362F
:10658000A3624035D4E90A239A4202D32046FFF79A
:1065900095FF8AF31188BD42D8D289F31188C9E7E3
:1065A00030465A46FBF7E4FAA36A5B445E44A362B2
:1065B0005D44E7E710B5029C0172043303FB04213C
:1065C000C0E906130023C0E90A33039B0363049B5D
:1065D000C460C0E90000C0E90422C0E90842436386
:1065E00010BD0000026AC260426AC0E904220022B3
:1065F000C0E90A226FF00101FEF77ABDD0E9042359
:106600009A4201D1C26822B9184650F8043B0B6087
:10661000704700231846FAE7C368C2690133C360B4
:106620004369134482694361934224BF436A4361CF
:106630000021FEF751BD000038B504460D46E36861
:106640003BB123691A1DA262E2691344E362002090
:1066500007E0237A33B929462046FEF72DFD0028AE
:10666000EDDA38BD6FF00100FBE700000369196047
:10667000C268013AC260C2691344826903619342ED
:1066800024BF436A036100238362036B03B118478D
:106690007047000070B530230D460446114683F361
:1066A0001188866A2EB9FFF7C7FF10B186F31188EB
:1066B00070BDA36A1D70A36AE26A01339342A362AC
:1066C00004D3E16920460439FFF7D0FF002080F3AE
:1066D0001188EDE72DE9F84F04460D46904699469E
:1066E0004FF0300A8AF311880026B346A76A4FB9E3
:1066F00049462046FFF7A0FF20B187F311883046B6
:10670000BDE8F88FD4E90A073A1AA8EB06079742C2
:1067100028BF1746402F1BD905F1400355F8042B1D
:1067200040F8042B9D42F9D1A36A4033A36240365E
:10673000D4E90A239A4204D3E16920460439FFF7D9
:1067400095FF8BF311884645D9D28AF31188CDE79E
:1067500029463A46FBF70CFAA36A3B443D44A36240
:106760003E44E5E7D0E904239A4217D1C3689BB1C0
:10677000836A8BB1043B9B1A0ED01360C368013B44
:10678000C360C3691A44836902619A4224BF436AA1
:106790000361002383620123184670470023FBE74F
:1067A00000F0D2B84FF08043586A70474FF08043F2
:1067B000002258631A610222DA6070474FF080436A
:1067C0000022DA60704700004FF080435863704742
:1067D000FEE7000070B51B4B01630025044686B040
:1067E000586085620E46FDF7DDFB04F11003C4E935
:1067F00004334FF0FF33C4E90635C4E90044A56013
:10680000E562FFF7CFFF2B460246C4E9082304F1F7
:1068100034010D4A256580232046FEF703FC012341
:10682000E0600A4A0375009272680192B268CDE98D
:106830000223074B6846CDE90435FEF71BFC06B082
:1068400070BD00BF60500020387200083D72000823
:10685000D1670008024AD36A1843D062704700BF6C
:10686000F84D00204B6843608B688360CB68C36041
:106870000B6943614B6903628B6943620B68036078
:106880007047000008B5264B26481A6940F2FF11F0
:106890000A431A611A6922F4FF7222F001021A6196
:1068A0001A691A6B0A431A631A6D0A431A651E4A5B
:1068B0001B6D1146FFF7D6FF02F11C0100F5806049
:1068C000FFF7D0FF02F1380100F58060FFF7CAFF43
:1068D00002F1540100F58060FFF7C4FF02F170017E
:1068E00000F58060FFF7BEFF02F18C0100F58060CB
:1068F000FFF7B8FF02F1A80100F58060FFF7B2FFD3
:1069000002F1C40100F58060FFF7ACFF02F1E00185
:1069100000F58060FFF7A6FFBDE8084000F090B8E2
:1069200000380240000002404472000808B500F040
:106930000BFAFEF72BFBFFF797F8BDE80840FEF7D0
:10694000C3BD0000704700000F4B1A6C42F00102FB
:106950001A641A6E42F001021A660C4A1B6E9368A2
:1069600043F0010393604FF0804353229A624FF04B
:10697000FF32DA6200229A615A63DA605A600122B9
:106980005A611A60704700BF00380240002004E0DE
:106990004FF0804208B51169D3680B40D9B2C943A2
:1069A0009B07116107D5302383F31188FEF714FB91
:1069B000002383F3118808BD1F4B1A696FEAC25286
:1069C0006FEAD2521A611A69C2F308021A614FF0D3
:1069D000FF301A695A69586100215A6959615A6928
:1069E0001A6A62F080521A621A6A02F080521A62BF
:1069F0001A6A5A6A58625A6A59625A6A1A6C42F09A
:106A000080521A641A6E42F080521A661A6E0B4A4D
:106A1000106840F480701060186F00F44070B0F59A
:106A2000007F1EBF4FF4803018671967536823F446
:106A30000073536000F060B90038024000700040FD
:106A4000344B4FF080521A64334A4FF44041116086
:106A50001A6842F001021A601A689107FCD59A6818
:106A600022F003029A602B4B9A6812F00C02FBD1C1
:106A7000196801F0F90119609A601A6842F48032CD
:106A80001A601A689203FCD55A6F42F001025A67E5
:106A9000204B5A6F9007FCD5204A5A601A6842F082
:106AA00080721A601C4A53685904FCD5194B1A6845
:106AB0009201FCD51A4A9A600322C3F88C20194B24
:106AC0001A68194B9A42194B21D1194A1168194A6F
:106AD00091421CD140F205121A60144A136803F067
:106AE0000F03052BFAD10B4B9A6842F002029A6011
:106AF0009A6802F00C02082AFAD15A6C42F48042D9
:106B00005A645A6E42F480425A665B6E704740F295
:106B10000572E1E700380240007000401854400759
:106B200000948838002004E011640020003C0240FA
:106B300000ED00E041C20F41074A08B5536903F078
:106B40000103536123B1054A13680BB1506898479C
:106B5000BDE80840FDF74ABA003C014080580020DB
:106B6000074A08B5536903F00203536123B1054A8C
:106B700093680BB1D0689847BDE80840FDF736BA76
:106B8000003C014080580020074A08B5536903F0D3
:106B90000403536123B1054A13690BB15069984747
:106BA000BDE80840FDF722BA003C014080580020B3
:106BB000074A08B5536903F00803536123B1054A36
:106BC00093690BB1D0699847BDE80840FDF70EBA4C
:106BD000003C014080580020074A08B5536903F083
:106BE0001003536123B1054A136A0BB1506A9847E9
:106BF000BDE80840FDF7FAB9003C0140805800208C
:106C0000164B10B55C6904F478725A61A30604D57A
:106C1000134A936A0BB1D06A9847600604D5104AAC
:106C2000136B0BB1506B9847210604D50C4A936B3C
:106C30000BB1D06B9847E20504D5094A136C0BB130
:106C4000506C9847A30504D5054A936C0BB1D06CE2
:106C50009847BDE81040FDF7C9B900BF003C0140AE
:106C600080580020194B10B55C6904F47C425A61CD
:106C7000620504D5164A136D0BB1506D9847230574
:106C800004D5134A936D0BB1D06D9847E00404D539
:106C90000F4A136E0BB1506E9847A10404D50C4AED
:106CA000936E0BB1D06E9847620404D5084A136FF7
:106CB0000BB1506F9847230404D5054A936F0BB16D
:106CC000D06F9847BDE81040FDF790B9003C0140F7
:106CD0008058002008B50348FDF724FABDE80840B5
:106CE000FDF784B9884B002008B5FFF751FEBDE8D9
:106CF0000840FDF77BB90000062108B50846FDF7FE
:106D000093FA06210720FDF78FFA06210820FDF7E8
:106D10008BFA06210920FDF787FA06210A20FDF7E4
:106D200083FA06211720FDF77FFA06212820FDF7B8
:106D30007BFA07211C20FDF777FABDE808400C21FB
:106D40002620FDF771BA000008B5FFF735FE00F008
:106D50000DF8FDF711FCFDF7F7FDFDF7CFFCFFF790
:106D6000F1FDBDE80840FFF71BBD00000023054A08
:106D700019460133102BC2E9001102F10802F8D1C3
:106D8000704700BF805800200B460146184600F0AF
:106D90002DB8000000F040B8012838BF012010B520
:106DA0000446204600F030F830B900F007F808B982
:106DB00000F00CF88047F4E710BD0000024B1868A3
:106DC000BFF35B8F704700BF0059002008B5062055
:106DD00000F084F80120FEF7C5FA0000024B0A46D5
:106DE00001461868FEF758BD5823002010B5054C21
:106DF00013462CB10A4601460220AFF3008010BDB5
:106E00002046FCE700000000024B01461868FEF730
:106E100047BD00BF58230020024B01461868FEF70B
:106E200043BD00BF5823002010B5013902449042F1
:106E300001D1002005E0037811F8014FA34201D0F1
:106E4000181B10BD0130F2E72DE9F041A3B1C91ABA
:106E500017780144044603F1FF3C8C42204601D9D7
:106E6000002009E00578BD4204F10104F5D10CEBE6
:106E70000405D618A54201D1BDE8F08115F8018DB1
:106E800016F801EDF045F5D0E7E700001F2938B509
:106E900004460D4604D9162303604FF0FF3038BD79
:106EA000426C12B152F821304BB9204600F030F854
:106EB0002A4601462046BDE8384000F017B8012BAD
:106EC0000AD0591C03D1162303600120E7E70024F0
:106ED00042F82540284698470020E0E7024B01464B
:106EE0001868FFF7D3BF00BF5823002038B5074DFF
:106EF00000230446084611462B60FEF737FA431C70
:106F000002D12B6803B1236038BD00BF04590020B3
:106F1000FEF726BA034611F8012B03F8012B002ACD
:106F2000F9D170476F72672E6172647570696C6F0A
:106F3000742E50697872616365722D706572697024
:106F40006800000053544D3332463F3F3F005354D6
:106F50004D3332463430780053544D333246343258
:106F6000780053544D3332463434365858000000BC
:106F7000012033000010410001105A000310590095
:106F80000710310000000000446F000813040000E7
:106F90004E6F000819040000586F0008210400001B
:106FA000626F000840A2E4F1646891060041A3E525
:106FB000F2656992070000004261642043414E4936
:106FC0006661636520696E6465782E00800000004C
:106FD00000800000000080000000000000000000B1
:106FE000F5240008DD2C00083D2C000805250008CC
:106FF000392500083527000809250008192500084B
:107000000D25000815250008112500085D2600083B
:107010001D250008A92F00082D250008312600088D
:1070200000960000000000000000000000000000CA
:107030000000000000000000394500082545000858
:10704000614500084D4500085945000845450008C0
:10705000314500081D4500086D450008000000008E
:107060007946000865460008A14600088D460008DC
:107070009946000885460008714600085D460008EC
:10708000AD46000800000000010000000000000004
:107090006330000090700008504E002060500020C7
:1070A0004172647550696C6F740025424F415244BF
:1070B000252D424C002553455249414C25000000E6
:1070C0000200000000000000954800080149000887
:1070D0004000400000550020105500200200000034
:1070E0000000000003000000000000004549000807
:1070F00000000000100000002055002000000000EB
:1071000001000000000000000858002001010200FA
:10711000655400087553000811540008F553000821
:10712000430000002871000809024300020100C06A
:1071300032090400000102020100052400100105CB
:10714000240100010424020205240600010705822F
:10715000030800FF09040100020A000000070501FE
:1071600002400000070581024000000012000000FC
:107170007471000812011001020000400912415709
:1071800000020102030100000403090425424F41EB
:1071900052442500303132333435363738394142A4
:1071A000434445460000000000400000004000004D
:1071B000004000000040000000000100000002004C
:1071C00000000200000002000000020000000200B7
:1071D000000002000000020000400000004000002B
:1071E000004000000040000000000100000002001C
:1071F0000000020000000200000002000000020087
:10720000000002000000020000000000894A00089F
:10721000414D0008ED4D0008400040006858002036
:10722000685800200100000078580020800000000D
:1072300040010000030000006D61696E0069646C2C
:10724000650000000000802A00000000AAAAAAAA87
:1072500000000024FFFF00000000000000A00A0062
:107260004400000000000000AAAAAAAA0000000032
:10727000FFFF0000000000000000000010000040C0
:1072800000000000AAAAAAAA10000040FFFF000008
:1072900000000000000000000A681000000000006C
:1072A000AAAAAAAA00541000FFFF000099007007C4
:1072B000000000000000004000000000AAAAAAAAE6
:1072C00000000040FFFF0000000000000000000080
:1072D0000000000000000000AAAAAAAA0000000006
:1072E000FFFF0000000000000000000000000000A0
:1072F00000000000AAAAAAAA00000000FFFF0000E8
:10730000000000000000000000000000000000007D
:107310000A00000000000000030000000000000060
:10732000000000000000000000000000000000005D
:10733000000000000000000000000000000000004D
:10734000E08EFF7F010000007A05000000000000D1
:1073500000001F000000000040420F00FE2A010054
:10736000D2040000FF00000068500020884B00207D
:1073700000960000000008009600000000080000D1
:1073800004000000887100080000000000000000F8
:1073900000000000000000000000000000000000ED
:1073A0005C2300200000000000000000000000003E
:1073B00000000000000000000000000000000000CD
:1073C00000000000000000000000000000000000BD
:1073D00000000000000000000000000000000000AD
:1073E000000000000000000000000000000000009D
:1073F000000000000000000000000000000000008D
:047400000000000088
:00000001FF
